 nio

 Timestamp is 4a75dac9 (reproducible build file hash)

 Preferred load address is 0000000180000000

 Start         Length     Name                   Class
 0001:00000000 000098f0H .text$mn                CODE
 0001:000098f0 00000036H .text$mn$00             CODE
 0001:00009926 00000092H .text$x                 CODE
 0002:00000000 00000620H .idata$5                DATA
 0002:00000620 00000038H .00cfg                  DATA
 0002:00000658 00000008H .CRT$XCA                DATA
 0002:00000660 00000008H .CRT$XCZ                DATA
 0002:00000668 00000008H .CRT$XIA                DATA
 0002:00000670 00000008H .CRT$XIZ                DATA
 0002:00000678 00000008H .CRT$XPA                DATA
 0002:00000680 00000008H .CRT$XPZ                DATA
 0002:00000688 00000008H .CRT$XTA                DATA
 0002:00000690 00000010H .CRT$XTZ                DATA
 0002:00000698 00000000H .gehcont$y              DATA
 0002:00000698 00000000H .gfids$y                DATA
 0002:000006a0 00000de0H .rdata                  DATA
 0002:00001480 00000000H .rdata$CastGuardVftablesA DATA
 0002:00001480 00000000H .rdata$CastGuardVftablesC DATA
 0002:00001480 0000008cH .rdata$voltmd           DATA
 0002:0000150c 000002b4H .rdata$zzzdbg           DATA
 0002:000017c0 00000008H .rtc$IAA                DATA
 0002:000017c8 00000008H .rtc$IZZ                DATA
 0002:000017d0 00000008H .rtc$TAA                DATA
 0002:000017d8 00000008H .rtc$TZZ                DATA
 0002:000017e0 00000880H .xdata                  DATA
 0002:00002060 00002e5cH .edata                  DATA
 0002:00004ebc 000000c8H .idata$2                DATA
 0002:00004f84 00000014H .idata$3                DATA
 0002:00004f98 00000620H .idata$4                DATA
 0002:000055b8 00000de4H .idata$6                DATA
 0003:00000000 00000230H .data                   DATA
 0003:00000230 000009e8H .bss                    DATA
 0004:00000000 00000aecH .pdata                  DATA
 0005:00000000 00000060H .rsrc$01                DATA
 0005:00000060 00000380H .rsrc$02                DATA

  Address         Publics by Value              Rva+Base               Lib:Object

 0000:00000000       __AbsoluteZero             0000000000000000     <absolute>
 0000:00000000       ___safe_se_handler_count   0000000000000000     <absolute>
 0000:00000000       ___safe_se_handler_table   0000000000000000     <absolute>
 0000:00000000       __arm64x_extra_rfe_table   0000000000000000     <absolute>
 0000:00000000       __arm64x_extra_rfe_table_size 0000000000000000     <absolute>
 0000:00000000       __arm64x_native_entrypoint 0000000000000000     <absolute>
 0000:00000000       __arm64x_redirection_metadata 0000000000000000     <absolute>
 0000:00000000       __arm64x_redirection_metadata_count 0000000000000000     <absolute>
 0000:00000000       __dynamic_value_reloc_table 0000000000000000     <absolute>
 0000:00000000       __enclave_config           0000000000000000     <absolute>
 0000:00000000       __guard_check_icall_a64n_fptr 0000000000000000     <absolute>
 0000:00000000       __guard_eh_cont_count      0000000000000000     <absolute>
 0000:00000000       __guard_eh_cont_table      0000000000000000     <absolute>
 0000:00000000       __guard_fids_count         0000000000000000     <absolute>
 0000:00000000       __guard_fids_table         0000000000000000     <absolute>
 0000:00000000       __guard_iat_count          0000000000000000     <absolute>
 0000:00000000       __guard_iat_table          0000000000000000     <absolute>
 0000:00000000       __guard_longjmp_count      0000000000000000     <absolute>
 0000:00000000       __guard_longjmp_table      0000000000000000     <absolute>
 0000:00000000       __hybrid_auxiliary_iat     0000000000000000     <absolute>
 0000:00000000       __hybrid_auxiliary_iat_copy 0000000000000000     <absolute>
 0000:00000000       __hybrid_code_map          0000000000000000     <absolute>
 0000:00000000       __hybrid_code_map_count    0000000000000000     <absolute>
 0000:00000000       __x64_code_ranges_to_entry_points 0000000000000000     <absolute>
 0000:00000000       __x64_code_ranges_to_entry_points_count 0000000000000000     <absolute>
 0000:00000100       __guard_flags              0000000000000100     <absolute>
 0000:00000000       __ImageBase                0000000180000000     <linker-defined>
 0001:00000000       Java_sun_nio_ch_DatagramChannelImpl_disconnect0 0000000180001000 f   DatagramChannelImpl.obj
 0001:000000c8       Java_sun_nio_ch_DatagramChannelImpl_receive0 00000001800010c8 f   DatagramChannelImpl.obj
 0001:000001ac       Java_sun_nio_ch_DatagramChannelImpl_send0 00000001800011ac f   DatagramChannelImpl.obj
 0001:0000022c       purgeOutstandingICMP       000000018000122c f   DatagramChannelImpl.obj
 0001:00000340       Java_sun_nio_ch_DatagramDispatcher_read0 0000000180001340 f   DatagramDispatcher.obj
 0001:00000438       Java_sun_nio_ch_DatagramDispatcher_readv0 0000000180001438 f   DatagramDispatcher.obj
 0001:00000590       Java_sun_nio_ch_DatagramDispatcher_write0 0000000180001590 f   DatagramDispatcher.obj
 0001:00000674       Java_sun_nio_ch_DatagramDispatcher_writev0 0000000180001674 f   DatagramDispatcher.obj
 0001:000007b4       Java_sun_nio_ch_FileDispatcherImpl_allocationGranularity0 00000001800017b4 f   FileDispatcherImpl.obj
 0001:000007d0       Java_sun_nio_ch_FileDispatcherImpl_available0 00000001800017d0 f   FileDispatcherImpl.obj
 0001:00000880       Java_sun_nio_ch_FileDispatcherImpl_close0 0000000180001880 f   FileDispatcherImpl.obj
 0001:000008bc       Java_sun_nio_ch_FileDispatcherImpl_duplicateHandle 00000001800018bc f   FileDispatcherImpl.obj
 0001:0000091c       Java_sun_nio_ch_FileDispatcherImpl_force0 000000018000191c f   FileDispatcherImpl.obj
 0001:0000097c       Java_sun_nio_ch_FileDispatcherImpl_isOther0 000000018000197c f   FileDispatcherImpl.obj
 0001:00000a98       Java_sun_nio_ch_FileDispatcherImpl_lock0 0000000180001a98 f   FileDispatcherImpl.obj
 0001:00000b84       Java_sun_nio_ch_FileDispatcherImpl_map0 0000000180001b84 f   FileDispatcherImpl.obj
 0001:00000cb8       Java_sun_nio_ch_FileDispatcherImpl_maxDirectTransferSize0 0000000180001cb8 f   FileDispatcherImpl.obj
 0001:00000cc0       Java_sun_nio_ch_FileDispatcherImpl_pread0 0000000180001cc0 f   FileDispatcherImpl.obj
 0001:00000de8       Java_sun_nio_ch_FileDispatcherImpl_pwrite0 0000000180001de8 f   FileDispatcherImpl.obj
 0001:00000ee8       Java_sun_nio_ch_FileDispatcherImpl_read0 0000000180001ee8 f   FileDispatcherImpl.obj
 0001:00000f8c       Java_sun_nio_ch_FileDispatcherImpl_readv0 0000000180001f8c f   FileDispatcherImpl.obj
 0001:00001080       Java_sun_nio_ch_FileDispatcherImpl_release0 0000000180002080 f   FileDispatcherImpl.obj
 0001:00001138       Java_sun_nio_ch_FileDispatcherImpl_seek0 0000000180002138 f   FileDispatcherImpl.obj
 0001:000011a0       Java_sun_nio_ch_FileDispatcherImpl_setDirect0 00000001800021a0 f   FileDispatcherImpl.obj
 0001:00001234       Java_sun_nio_ch_FileDispatcherImpl_size0 0000000180002234 f   FileDispatcherImpl.obj
 0001:0000127c       Java_sun_nio_ch_FileDispatcherImpl_transferTo0 000000018000227c f   FileDispatcherImpl.obj
 0001:00001374       Java_sun_nio_ch_FileDispatcherImpl_truncate0 0000000180002374 f   FileDispatcherImpl.obj
 0001:000013d0       Java_sun_nio_ch_FileDispatcherImpl_unmap0 00000001800023d0 f   FileDispatcherImpl.obj
 0001:00001404       Java_sun_nio_ch_FileDispatcherImpl_write0 0000000180002404 f   FileDispatcherImpl.obj
 0001:000014c4       Java_sun_nio_ch_FileDispatcherImpl_writev0 00000001800024c4 f   FileDispatcherImpl.obj
 0001:000015d4       Java_sun_nio_ch_FileKey_init 00000001800025d4 f   FileKey.obj
 0001:0000167c       Java_sun_nio_ch_IOUtil_configureBlocking 000000018000267c f   IOUtil.obj
 0001:000016e8       Java_sun_nio_ch_IOUtil_drain 00000001800026e8 f   IOUtil.obj
 0001:00001774       Java_sun_nio_ch_IOUtil_fdVal 0000000180002774 f   IOUtil.obj
 0001:00001788       Java_sun_nio_ch_IOUtil_initIDs 0000000180002788 f   IOUtil.obj
 0001:00001804       Java_sun_nio_ch_IOUtil_iovMax 0000000180002804 f   IOUtil.obj
 0001:00001804       Java_sun_nio_ch_NativeSocketAddress_sizeofSockAddr4 0000000180002804 f   NativeSocketAddress.obj
 0001:00001804       Java_sun_nio_ch_Net_pollconnValue 0000000180002804 f   Net.obj
 0001:00001804       Java_sun_nio_ch_Net_polloutValue 0000000180002804 f   Net.obj
 0001:00001804       Java_sun_nio_ch_WEPoll_eventSize 0000000180002804 f   WEPollNatives.obj
 0001:0000180c       Java_sun_nio_ch_IOUtil_randomBytes 000000018000280c f   IOUtil.obj
 0001:00001814       Java_sun_nio_ch_IOUtil_setfdVal 0000000180002814 f   IOUtil.obj
 0001:00001828       Java_sun_nio_ch_IOUtil_write1 0000000180002828 f   IOUtil.obj
 0001:0000188c       Java_sun_nio_ch_IOUtil_writevMax 000000018000288c f   IOUtil.obj
 0001:00001898       convertLongReturnVal       0000000180002898 f   IOUtil.obj
 0001:000018c8       convertReturnVal           00000001800028c8 f   IOUtil.obj
 0001:000018f4       fdval                      00000001800028f4 f   IOUtil.obj
 0001:00001908       handleval                  0000000180002908 f   IOUtil.obj
 0001:0000191c       setfdval                   000000018000291c f   IOUtil.obj
 0001:00001930       Java_sun_nio_ch_Iocp_close0 0000000180002930 f   Iocp.obj
 0001:00001930       Java_sun_nio_fs_WindowsNativeDispatcher_CloseHandle 0000000180002930 f   WindowsNativeDispatcher.obj
 0001:0000193c       Java_sun_nio_ch_Iocp_createIoCompletionPort 000000018000293c f   Iocp.obj
 0001:00001988       Java_sun_nio_ch_Iocp_getErrorMessage 0000000180002988 f   Iocp.obj
 0001:00001988       Java_sun_nio_fs_WindowsNativeDispatcher_FormatMessage 0000000180002988 f   WindowsNativeDispatcher.obj
 0001:00001a64       Java_sun_nio_ch_Iocp_getQueuedCompletionStatus 0000000180002a64 f   Iocp.obj
 0001:00001b30       Java_sun_nio_ch_Iocp_initIDs 0000000180002b30 f   Iocp.obj
 0001:00001c04       Java_sun_nio_ch_Iocp_postQueuedCompletionStatus 0000000180002c04 f   Iocp.obj
 0001:00001c3c       Java_sun_nio_ch_Net_canJoin6WithIPv4Group0 0000000180002c3c f   Net.obj
 0001:00001c3c       Java_sun_nio_ch_Net_canUseIPv6OptionsWithIPv4LocalAddress0 0000000180002c3c f   Net.obj
 0001:00001c3c       Java_sun_nio_ch_Net_isReusePortAvailable0 0000000180002c3c f   Net.obj
 0001:00001c3c       MappedMemoryUtils_isLoaded0 0000000180002c3c f   MappedMemoryUtils.obj
 0001:00001c40       MappedMemoryUtils_load0    0000000180002c40 f   MappedMemoryUtils.obj
 0001:00001c40       MappedMemoryUtils_unload0  0000000180002c40 f   MappedMemoryUtils.obj
 0001:00001c40       _guard_check_icall_nop     0000000180002c40 f   MSVCRT:guard_support.obj
 0001:00001c44       MappedMemoryUtils_force0   0000000180002c44 f   MappedMemoryUtils.obj
 0001:00001d30       Java_java_nio_MappedMemoryUtils_registerNatives 0000000180002d30 f   MappedMemoryUtils.obj
 0001:00001d48       Java_sun_nio_ch_NativeSocketAddress_AFINET 0000000180002d48 f   NativeSocketAddress.obj
 0001:00001d48       Java_sun_nio_ch_NativeSocketAddress_offsetSin4Port 0000000180002d48 f   NativeSocketAddress.obj
 0001:00001d48       Java_sun_nio_ch_NativeSocketAddress_offsetSin6Port 0000000180002d48 f   NativeSocketAddress.obj
 0001:00001d48       Java_sun_nio_ch_NativeSocketAddress_sizeofFamily 0000000180002d48 f   NativeSocketAddress.obj
 0001:00001d48       Java_sun_nio_ch_Net_pollhupValue 0000000180002d48 f   Net.obj
 0001:00001d50       Java_sun_nio_ch_NativeSocketAddress_AFINET6 0000000180002d50 f   NativeSocketAddress.obj
 0001:00001d58       Java_sun_nio_ch_NativeSocketAddress_offsetFamily 0000000180002d58 f   NativeSocketAddress.obj
 0001:00001d58       Java_sun_nio_ch_WEPoll_eventsOffset 0000000180002d58 f   WEPollNatives.obj
 0001:00001d58       __scrt_stub_for_is_c_termination_complete 0000000180002d58 f   MSVCRT:ucrt_stubs.obj
 0001:00001d58       _is_c_termination_complete 0000000180002d58 f   MSVCRT:ucrt_stubs.obj
 0001:00001d5c       Java_sun_nio_ch_NativeSocketAddress_offsetSin4Addr 0000000180002d5c f   NativeSocketAddress.obj
 0001:00001d5c       Java_sun_nio_ch_NativeSocketAddress_offsetSin6FlowInfo 0000000180002d5c f   NativeSocketAddress.obj
 0001:00001d5c       Java_sun_nio_ch_Net_pollnvalValue 0000000180002d5c f   Net.obj
 0001:00001d64       Java_sun_nio_ch_NativeSocketAddress_offsetSin6Addr 0000000180002d64 f   NativeSocketAddress.obj
 0001:00001d64       Java_sun_nio_ch_WEPoll_dataOffset 0000000180002d64 f   WEPollNatives.obj
 0001:00001d6c       Java_sun_nio_ch_NativeSocketAddress_offsetSin6ScopeId 0000000180002d6c f   NativeSocketAddress.obj
 0001:00001d74       Java_sun_nio_ch_NativeSocketAddress_sizeofSockAddr6 0000000180002d74 f   NativeSocketAddress.obj
 0001:00001d7c       Java_sun_nio_ch_Net_accept 0000000180002d7c f   Net.obj
 0001:00001eb0       Java_sun_nio_ch_Net_available 0000000180002eb0 f   Net.obj
 0001:00001f04       Java_sun_nio_ch_Net_bind0  0000000180002f04 f   Net.obj
 0001:00001fac       Java_sun_nio_ch_Net_blockOrUnblock4 0000000180002fac f   Net.obj
 0001:00002084       Java_sun_nio_ch_Net_blockOrUnblock6 0000000180003084 f   Net.obj
 0001:000020dc       Java_sun_nio_ch_Net_canIPv6SocketJoinIPv4Group0 00000001800030dc f   Net.obj
 0001:000020dc       Java_sun_nio_ch_Net_shouldSetBothIPv4AndIPv6Options0 00000001800030dc f   Net.obj
 0001:000020dc       Java_sun_nio_ch_Net_shouldShutdownWriteBeforeClose0 00000001800030dc f   Net.obj
 0001:000020dc       __acrt_initialize          00000001800030dc f   MSVCRT:ucrt_stubs.obj
 0001:000020dc       __acrt_thread_attach       00000001800030dc f   MSVCRT:ucrt_stubs.obj
 0001:000020dc       __acrt_thread_detach       00000001800030dc f   MSVCRT:ucrt_stubs.obj
 0001:000020dc       __acrt_uninitialize        00000001800030dc f   MSVCRT:ucrt_stubs.obj
 0001:000020dc       __acrt_uninitialize_critical 00000001800030dc f   MSVCRT:ucrt_stubs.obj
 0001:000020dc       __scrt_stub_for_acrt_initialize 00000001800030dc f   MSVCRT:ucrt_stubs.obj
 0001:000020dc       __scrt_stub_for_acrt_thread_attach 00000001800030dc f   MSVCRT:ucrt_stubs.obj
 0001:000020dc       __scrt_stub_for_acrt_thread_detach 00000001800030dc f   MSVCRT:ucrt_stubs.obj
 0001:000020dc       __scrt_stub_for_acrt_uninitialize 00000001800030dc f   MSVCRT:ucrt_stubs.obj
 0001:000020dc       __scrt_stub_for_acrt_uninitialize_critical 00000001800030dc f   MSVCRT:ucrt_stubs.obj
 0001:000020dc       __vcrt_initialize          00000001800030dc f   MSVCRT:ucrt_stubs.obj
 0001:000020dc       __vcrt_thread_attach       00000001800030dc f   MSVCRT:ucrt_stubs.obj
 0001:000020dc       __vcrt_thread_detach       00000001800030dc f   MSVCRT:ucrt_stubs.obj
 0001:000020dc       __vcrt_uninitialize        00000001800030dc f   MSVCRT:ucrt_stubs.obj
 0001:000020dc       __vcrt_uninitialize_critical 00000001800030dc f   MSVCRT:ucrt_stubs.obj
 0001:000020e0       Java_sun_nio_ch_Net_connect0 00000001800030e0 f   Net.obj
 0001:00002400       Java_sun_nio_ch_Net_discardOOB 0000000180003400 f   Net.obj
 0001:000024a0       Java_sun_nio_ch_Net_getIntOption0 00000001800034a0 f   Net.obj
 0001:000025c0       Java_sun_nio_ch_Net_getInterface4 00000001800035c0 f   Net.obj
 0001:0000262c       Java_sun_nio_ch_Net_getInterface6 000000018000362c f   Net.obj
 0001:00002694       Java_sun_nio_ch_Net_initIDs 0000000180003694 f   Net.obj
 0001:00002718       Java_sun_nio_ch_Net_isExclusiveBindAvailable 0000000180003718 f   Net.obj
 0001:00002718       Java_sun_nio_ch_Net_pollerrValue 0000000180003718 f   Net.obj
 0001:00002718       _get_startup_argv_mode     0000000180003718 f   MSVCRT:argv_mode.obj
 0001:00002720       Java_sun_nio_ch_Net_isIPv6Available0 0000000180003720 f   Net.obj
 0001:00002734       Java_sun_nio_ch_Net_joinOrDrop4 0000000180003734 f   Net.obj
 0001:00002850       Java_sun_nio_ch_Net_joinOrDrop6 0000000180003850 f   Net.obj
 0001:0000293c       Java_sun_nio_ch_Net_listen 000000018000393c f   Net.obj
 0001:00002994       Java_sun_nio_ch_Net_localInetAddress 0000000180003994 f   Net.obj
 0001:00002a14       Java_sun_nio_ch_Net_localPort 0000000180003a14 f   Net.obj
 0001:00002a9c       Java_sun_nio_ch_Net_poll   0000000180003a9c f   Net.obj
 0001:00002c38       Java_sun_nio_ch_Net_pollConnect 0000000180003c38 f   Net.obj
 0001:00002db8       Java_sun_nio_ch_Net_pollinValue 0000000180003db8 f   Net.obj
 0001:00002dc0       Java_sun_nio_ch_Net_remoteInetAddress 0000000180003dc0 f   Net.obj
 0001:00002e40       Java_sun_nio_ch_Net_remotePort 0000000180003e40 f   Net.obj
 0001:00002ec8       Java_sun_nio_ch_Net_sendOOB 0000000180003ec8 f   Net.obj
 0001:00002f28       Java_sun_nio_ch_Net_setIntOption0 0000000180003f28 f   Net.obj
 0001:00002ffc       Java_sun_nio_ch_Net_setInterface4 0000000180003ffc f   Net.obj
 0001:00003068       Java_sun_nio_ch_Net_setInterface6 0000000180004068 f   Net.obj
 0001:000030c0       Java_sun_nio_ch_Net_shutdown 00000001800040c0 f   Net.obj
 0001:0000311c       Java_sun_nio_ch_Net_socket0 000000018000411c f   Net.obj
 0001:00003340       Java_sun_nio_fs_RegistryFileTypeDetector_queryStringValue 0000000180004340 f   RegistryFileTypeDetector.obj
 0001:00003418       Java_sun_nio_ch_SocketDispatcher_close0 0000000180004418 f   SocketDispatcher.obj
 0001:00003480       Java_sun_nio_ch_SocketDispatcher_read0 0000000180004480 f   SocketDispatcher.obj
 0001:0000355c       Java_sun_nio_ch_SocketDispatcher_readv0 000000018000455c f   SocketDispatcher.obj
 0001:000036bc       Java_sun_nio_ch_SocketDispatcher_write0 00000001800046bc f   SocketDispatcher.obj
 0001:000037ac       Java_sun_nio_ch_SocketDispatcher_writev0 00000001800047ac f   SocketDispatcher.obj
 0001:00003948       Java_sun_nio_ch_UnixDomainSockets_accept0 0000000180004948 f   UnixDomainSockets.obj
 0001:00003a54       Java_sun_nio_ch_UnixDomainSockets_bind0 0000000180004a54 f   UnixDomainSockets.obj
 0001:00003af0       Java_sun_nio_ch_UnixDomainSockets_connect0 0000000180004af0 f   UnixDomainSockets.obj
 0001:00003bec       Java_sun_nio_ch_UnixDomainSockets_init 0000000180004bec f   UnixDomainSockets.obj
 0001:00003e28       Java_sun_nio_ch_UnixDomainSockets_localAddress0 0000000180004e28 f   UnixDomainSockets.obj
 0001:00003eac       Java_sun_nio_ch_UnixDomainSockets_socket0 0000000180004eac f   UnixDomainSockets.obj
 0001:00003f20       sockaddrToUnixAddressBytes 0000000180004f20 f   UnixDomainSockets.obj
 0001:00003fac       unixSocketAddressToSockaddr 0000000180004fac f   UnixDomainSockets.obj
 0001:000040ac       Java_sun_nio_ch_WEPoll_close 00000001800050ac f   WEPollNatives.obj
 0001:000040b4       Java_sun_nio_ch_WEPoll_create 00000001800050b4 f   WEPollNatives.obj
 0001:000040f0       Java_sun_nio_ch_WEPoll_ctl 00000001800050f0 f   WEPollNatives.obj
 0001:0000412c       Java_sun_nio_ch_WEPoll_wait 000000018000512c f   WEPollNatives.obj
 0001:0000416c       Java_sun_nio_ch_WindowsAsynchronousFileChannelImpl_lockFile 000000018000516c f   WindowsAsynchronousFileChannelImpl.obj
 0001:00004200       Java_sun_nio_ch_WindowsAsynchronousFileChannelImpl_readFile 0000000180005200 f   WindowsAsynchronousFileChannelImpl.obj
 0001:00004280       Java_sun_nio_ch_WindowsAsynchronousFileChannelImpl_writeFile 0000000180005280 f   WindowsAsynchronousFileChannelImpl.obj
 0001:000042f4       Java_sun_nio_ch_WindowsAsynchronousServerSocketChannelImpl_accept0 00000001800052f4 f   WindowsAsynchronousServerSocketChannelImpl.obj
 0001:000043a0       Java_sun_nio_ch_WindowsAsynchronousServerSocketChannelImpl_closesocket0 00000001800053a0 f   WindowsAsynchronousServerSocketChannelImpl.obj
 0001:000043a0       Java_sun_nio_ch_WindowsAsynchronousSocketChannelImpl_closesocket0 00000001800053a0 f   WindowsAsynchronousSocketChannelImpl.obj
 0001:000043cc       Java_sun_nio_ch_WindowsAsynchronousServerSocketChannelImpl_initIDs 00000001800053cc f   WindowsAsynchronousServerSocketChannelImpl.obj
 0001:000044d8       Java_sun_nio_ch_WindowsAsynchronousServerSocketChannelImpl_updateAcceptContext 00000001800054d8 f   WindowsAsynchronousServerSocketChannelImpl.obj
 0001:00004524       Java_sun_nio_ch_WindowsAsynchronousSocketChannelImpl_connect0 0000000180005524 f   WindowsAsynchronousSocketChannelImpl.obj
 0001:000045f4       Java_sun_nio_ch_WindowsAsynchronousSocketChannelImpl_initIDs 00000001800055f4 f   WindowsAsynchronousSocketChannelImpl.obj
 0001:00004700       Java_sun_nio_ch_WindowsAsynchronousSocketChannelImpl_read0 0000000180005700 f   WindowsAsynchronousSocketChannelImpl.obj
 0001:000047ac       Java_sun_nio_ch_WindowsAsynchronousSocketChannelImpl_shutdown0 00000001800057ac f   WindowsAsynchronousSocketChannelImpl.obj
 0001:000047dc       Java_sun_nio_ch_WindowsAsynchronousSocketChannelImpl_updateConnectContext 00000001800057dc f   WindowsAsynchronousSocketChannelImpl.obj
 0001:00004820       Java_sun_nio_ch_WindowsAsynchronousSocketChannelImpl_write0 0000000180005820 f   WindowsAsynchronousSocketChannelImpl.obj
 0001:000048c4       Java_sun_nio_fs_WindowsNativeDispatcher_AccessCheck 00000001800058c4 f   WindowsNativeDispatcher.obj
 0001:000049a4       Java_sun_nio_fs_WindowsNativeDispatcher_AddAccessAllowedAceEx 00000001800059a4 f   WindowsNativeDispatcher.obj
 0001:000049f0       Java_sun_nio_fs_WindowsNativeDispatcher_AddAccessDeniedAceEx 00000001800059f0 f   WindowsNativeDispatcher.obj
 0001:00004a3c       Java_sun_nio_fs_WindowsNativeDispatcher_AdjustTokenPrivileges 0000000180005a3c f   WindowsNativeDispatcher.obj
 0001:00004ab8       Java_sun_nio_fs_WindowsNativeDispatcher_CancelIo 0000000180005ab8 f   WindowsNativeDispatcher.obj
 0001:00004ae4       Java_sun_nio_fs_WindowsNativeDispatcher_ConvertSidToStringSid 0000000180005ae4 f   WindowsNativeDispatcher.obj
 0001:00004b54       Java_sun_nio_fs_WindowsNativeDispatcher_ConvertStringSidToSid0 0000000180005b54 f   WindowsNativeDispatcher.obj
 0001:00004b8c       Java_sun_nio_fs_WindowsNativeDispatcher_CopyFileEx0 0000000180005b8c f   WindowsNativeDispatcher.obj
 0001:00004bd8       Java_sun_nio_fs_WindowsNativeDispatcher_CreateDirectory0 0000000180005bd8 f   WindowsNativeDispatcher.obj
 0001:00004c24       Java_sun_nio_fs_WindowsNativeDispatcher_CreateEvent 0000000180005c24 f   WindowsNativeDispatcher.obj
 0001:00004c6c       Java_sun_nio_fs_WindowsNativeDispatcher_CreateFile0 0000000180005c6c f   WindowsNativeDispatcher.obj
 0001:00004d00       Java_sun_nio_fs_WindowsNativeDispatcher_CreateHardLink0 0000000180005d00 f   WindowsNativeDispatcher.obj
 0001:00004d38       Java_sun_nio_fs_WindowsNativeDispatcher_CreateIoCompletionPort 0000000180005d38 f   WindowsNativeDispatcher.obj
 0001:00004d84       Java_sun_nio_fs_WindowsNativeDispatcher_CreateSymbolicLink0 0000000180005d84 f   WindowsNativeDispatcher.obj
 0001:00004dbc       Java_sun_nio_fs_WindowsNativeDispatcher_DeleteFile0 0000000180005dbc f   WindowsNativeDispatcher.obj
 0001:00004de8       Java_sun_nio_fs_WindowsNativeDispatcher_DeviceIoControlGetReparsePoint 0000000180005de8 f   WindowsNativeDispatcher.obj
 0001:00004e40       Java_sun_nio_fs_WindowsNativeDispatcher_DeviceIoControlSetSparse 0000000180005e40 f   WindowsNativeDispatcher.obj
 0001:00004e94       Java_sun_nio_fs_WindowsNativeDispatcher_DuplicateTokenEx 0000000180005e94 f   WindowsNativeDispatcher.obj
 0001:00004ee4       Java_sun_nio_fs_WindowsNativeDispatcher_FindClose 0000000180005ee4 f   WindowsNativeDispatcher.obj
 0001:00004f10       Java_sun_nio_fs_WindowsNativeDispatcher_FindFirstFile0 0000000180005f10 f   WindowsNativeDispatcher.obj
 0001:00005008       Java_sun_nio_fs_WindowsNativeDispatcher_FindFirstFile1 0000000180006008 f   WindowsNativeDispatcher.obj
 0001:00005048       Java_sun_nio_fs_WindowsNativeDispatcher_FindFirstStream0 0000000180006048 f   WindowsNativeDispatcher.obj
 0001:00005150       Java_sun_nio_fs_WindowsNativeDispatcher_FindNextFile0 0000000180006150 f   WindowsNativeDispatcher.obj
 0001:000051c4       Java_sun_nio_fs_WindowsNativeDispatcher_FindNextStream0 00000001800061c4 f   WindowsNativeDispatcher.obj
 0001:00005258       Java_sun_nio_fs_WindowsNativeDispatcher_GetAce 0000000180006258 f   WindowsNativeDispatcher.obj
 0001:00005298       Java_sun_nio_fs_WindowsNativeDispatcher_GetAclInformation0 0000000180006298 f   WindowsNativeDispatcher.obj
 0001:0000531c       Java_sun_nio_fs_WindowsNativeDispatcher_GetCurrentProcess 000000018000631c f   WindowsNativeDispatcher.obj
 0001:00005324       Java_sun_nio_fs_WindowsNativeDispatcher_GetCurrentThread 0000000180006324 f   WindowsNativeDispatcher.obj
 0001:0000532c       Java_sun_nio_fs_WindowsNativeDispatcher_GetDiskFreeSpace0 000000018000632c f   WindowsNativeDispatcher.obj
 0001:0000539c       Java_sun_nio_fs_WindowsNativeDispatcher_GetDiskFreeSpaceEx0 000000018000639c f   WindowsNativeDispatcher.obj
 0001:00005438       Java_sun_nio_fs_WindowsNativeDispatcher_GetDriveType0 0000000180006438 f   WindowsNativeDispatcher.obj
 0001:00005444       Java_sun_nio_fs_WindowsNativeDispatcher_GetFileAttributes0 0000000180006444 f   WindowsNativeDispatcher.obj
 0001:00005480       Java_sun_nio_fs_WindowsNativeDispatcher_GetFileAttributesEx0 0000000180006480 f   WindowsNativeDispatcher.obj
 0001:000054b4       Java_sun_nio_fs_WindowsNativeDispatcher_GetFileInformationByHandle0 00000001800064b4 f   WindowsNativeDispatcher.obj
 0001:000054e4       Java_sun_nio_fs_WindowsNativeDispatcher_GetFileInformationByName0 00000001800064e4 f   WindowsNativeDispatcher.obj
 0001:0000553c       Java_sun_nio_fs_WindowsNativeDispatcher_GetFileSecurity0 000000018000653c f   WindowsNativeDispatcher.obj
 0001:000055a0       Java_sun_nio_fs_WindowsNativeDispatcher_GetFileSizeEx 00000001800065a0 f   WindowsNativeDispatcher.obj
 0001:000055d8       Java_sun_nio_fs_WindowsNativeDispatcher_GetFinalPathNameByHandle 00000001800065d8 f   WindowsNativeDispatcher.obj
 0001:000056f0       Java_sun_nio_fs_WindowsNativeDispatcher_GetFullPathName0 00000001800066f0 f   WindowsNativeDispatcher.obj
 0001:00005804       Java_sun_nio_fs_WindowsNativeDispatcher_GetLengthSid 0000000180006804 f   WindowsNativeDispatcher.obj
 0001:00005810       Java_sun_nio_fs_WindowsNativeDispatcher_GetLogicalDrives 0000000180006810 f   WindowsNativeDispatcher.obj
 0001:00005848       Java_sun_nio_fs_WindowsNativeDispatcher_GetOverlappedResult 0000000180006848 f   WindowsNativeDispatcher.obj
 0001:00005890       Java_sun_nio_fs_WindowsNativeDispatcher_GetQueuedCompletionStatus0 0000000180006890 f   WindowsNativeDispatcher.obj
 0001:00005940       Java_sun_nio_fs_WindowsNativeDispatcher_GetSecurityDescriptorDacl 0000000180006940 f   WindowsNativeDispatcher.obj
 0001:00005990       Java_sun_nio_fs_WindowsNativeDispatcher_GetSecurityDescriptorOwner 0000000180006990 f   WindowsNativeDispatcher.obj
 0001:000059d0       Java_sun_nio_fs_WindowsNativeDispatcher_GetTokenInformation 00000001800069d0 f   WindowsNativeDispatcher.obj
 0001:00005a30       Java_sun_nio_fs_WindowsNativeDispatcher_GetVolumeInformation0 0000000180006a30 f   WindowsNativeDispatcher.obj
 0001:00005b88       Java_sun_nio_fs_WindowsNativeDispatcher_GetVolumePathName0 0000000180006b88 f   WindowsNativeDispatcher.obj
 0001:00005c1c       Java_sun_nio_fs_WindowsNativeDispatcher_InitializeAcl 0000000180006c1c f   WindowsNativeDispatcher.obj
 0001:00005c54       Java_sun_nio_fs_WindowsNativeDispatcher_InitializeSecurityDescriptor 0000000180006c54 f   WindowsNativeDispatcher.obj
 0001:00005c88       Java_sun_nio_fs_WindowsNativeDispatcher_LocalFree 0000000180006c88 f   WindowsNativeDispatcher.obj
 0001:00005c94       Java_sun_nio_fs_WindowsNativeDispatcher_LookupAccountName0 0000000180006c94 f   WindowsNativeDispatcher.obj
 0001:00005d30       Java_sun_nio_fs_WindowsNativeDispatcher_LookupAccountSid0 0000000180006d30 f   WindowsNativeDispatcher.obj
 0001:00005e78       Java_sun_nio_fs_WindowsNativeDispatcher_LookupPrivilegeValue0 0000000180006e78 f   WindowsNativeDispatcher.obj
 0001:00005ef4       Java_sun_nio_fs_WindowsNativeDispatcher_MoveFileEx0 0000000180006ef4 f   WindowsNativeDispatcher.obj
 0001:00005f2c       Java_sun_nio_fs_WindowsNativeDispatcher_OpenProcessToken 0000000180006f2c f   WindowsNativeDispatcher.obj
 0001:00005f68       Java_sun_nio_fs_WindowsNativeDispatcher_OpenThreadToken 0000000180006f68 f   WindowsNativeDispatcher.obj
 0001:00005fc4       Java_sun_nio_fs_WindowsNativeDispatcher_PostQueuedCompletionStatus 0000000180006fc4 f   WindowsNativeDispatcher.obj
 0001:00006000       Java_sun_nio_fs_WindowsNativeDispatcher_ReadDirectoryChangesW 0000000180007000 f   WindowsNativeDispatcher.obj
 0001:00006070       Java_sun_nio_fs_WindowsNativeDispatcher_RemoveDirectory0 0000000180007070 f   WindowsNativeDispatcher.obj
 0001:0000609c       Java_sun_nio_fs_WindowsNativeDispatcher_SetEndOfFile 000000018000709c f   WindowsNativeDispatcher.obj
 0001:000060c8       Java_sun_nio_fs_WindowsNativeDispatcher_SetFileAttributes0 00000001800070c8 f   WindowsNativeDispatcher.obj
 0001:000060f8       Java_sun_nio_fs_WindowsNativeDispatcher_SetFileSecurity0 00000001800070f8 f   WindowsNativeDispatcher.obj
 0001:00006130       Java_sun_nio_fs_WindowsNativeDispatcher_SetFileTime0 0000000180007130 f   WindowsNativeDispatcher.obj
 0001:0000619c       Java_sun_nio_fs_WindowsNativeDispatcher_SetSecurityDescriptorDacl 000000018000719c f   WindowsNativeDispatcher.obj
 0001:000061d8       Java_sun_nio_fs_WindowsNativeDispatcher_SetSecurityDescriptorOwner 00000001800071d8 f   WindowsNativeDispatcher.obj
 0001:00006210       Java_sun_nio_fs_WindowsNativeDispatcher_SetThreadToken 0000000180007210 f   WindowsNativeDispatcher.obj
 0001:00006240       Java_sun_nio_fs_WindowsNativeDispatcher_init 0000000180007240 f   WindowsNativeDispatcher.obj
 0001:000066e8       Java_sun_nio_ch_WindowsSelectorImpl_00024SubSelector_poll0 00000001800076e8 f   WindowsSelectorImpl.obj
 0001:000069c8       Java_sun_nio_ch_WindowsSelectorImpl_resetWakeupSocket0 00000001800079c8 f   WindowsSelectorImpl.obj
 0001:00006a80       Java_sun_nio_ch_WindowsSelectorImpl_setWakeupSocket0 0000000180007a80 f   WindowsSelectorImpl.obj
 0001:00006aa4       JNI_OnLoad                 0000000180007aa4 f   nio_util.obj
 0001:00006c9c       epoll_close                0000000180007c9c f   wepoll.obj
 0001:00006dcc       epoll_create1              0000000180007dcc f   wepoll.obj
 0001:00006df0       epoll_ctl                  0000000180007df0 f   wepoll.obj
 0001:00006ec4       epoll_wait                 0000000180007ec4 f   wepoll.obj
 0001:00008933       JNU_ThrowByName            0000000180009933 f   java:java.dll
 0001:00008939       JNU_ThrowOutOfMemoryError  0000000180009939 f   java:java.dll
 0001:0000893f       JNU_ThrowIOExceptionWithLastError 000000018000993f f   java:java.dll
 0001:00008945       JNU_ThrowInternalError     0000000180009945 f   java:java.dll
 0001:0000894b       JNU_ThrowIOException       000000018000994b f   java:java.dll
 0001:00008951       Java_sun_security_provider_NativeSeedGenerator_nativeGenerateSeed 0000000180009951 f   java:java.dll
 0001:00008957       JNU_NewObjectByName        0000000180009957 f   java:java.dll
 0001:0000895d       NET_ThrowNew               000000018000995d f   net:net.dll
 0001:00008963       NET_WinBind                0000000180009963 f   net:net.dll
 0001:00008969       NET_EnableFastTcpLoopbackConnect 0000000180009969 f   net:net.dll
 0001:0000896f       initInetAddressIDs         000000018000996f f   net:net.dll
 0001:00008975       ipv6_available             0000000180009975 f   net:net.dll
 0001:0000897b       NET_InetAddressToSockaddr  000000018000997b f   net:net.dll
 0001:00008981       NET_SockaddrToInetAddress  0000000180009981 f   net:net.dll
 0001:00008987       NET_GetPortFromSockaddr    0000000180009987 f   net:net.dll
 0001:0000898d       NET_GetSockOpt             000000018000998d f   net:net.dll
 0001:00008993       NET_SetSockOpt             0000000180009993 f   net:net.dll
 0001:00008999       NET_EnableFastTcpLoopback  0000000180009999 f   net:net.dll
 0001:0000899f       ConvertSidToStringSidW     000000018000999f f   advapi32:ADVAPI32.dll
 0001:000089a5       ConvertStringSidToSidW     00000001800099a5 f   advapi32:ADVAPI32.dll
 0001:000089ab       TransmitFile               00000001800099ab f   mswsock:MSWSOCK.dll
 0001:000089b1       __WSAFDIsSet               00000001800099b1 f   ws2_32:WS2_32.dll
 0001:000089b7       inet_ntop                  00000001800099b7 f   ws2_32:WS2_32.dll
 0001:000089c0       __GSHandlerCheck           00000001800099c0 f   MSVCRT:gshandler.obj
 0001:000089e0       __GSHandlerCheckCommon     00000001800099e0 f   MSVCRT:gshandler.obj
 0001:00008a50       __security_check_cookie    0000000180009a50 f   MSVCRT:amdsecgs.obj
 0001:00008a70       __raise_securityfailure    0000000180009a70 f   MSVCRT:gs_report.obj
 0001:00008aa4       __report_gsfailure         0000000180009aa4 f   MSVCRT:gs_report.obj
 0001:00008b78       __report_rangecheckfailure 0000000180009b78 f   MSVCRT:gs_report.obj
 0001:00008b8c       __report_securityfailure   0000000180009b8c f   MSVCRT:gs_report.obj
 0001:00008d20       __chkstk                   0000000180009d20 f   MSVCRT:chkstk.obj
 0001:00008d20       _alloca_probe              0000000180009d20 f   MSVCRT:chkstk.obj
 0001:00009090       _DllMainCRTStartup         000000018000a090 f   MSVCRT:dll_dllmain.obj
 0001:000090d0       __security_init_cookie     000000018000a0d0 f   MSVCRT:gs_support.obj
 0001:0000917c       DllMain                    000000018000a17c f   MSVCRT:dll_dllmain_stub.obj
 0001:000091a0       ?__scrt_initialize_type_info@@YAXXZ 000000018000a1a0 f   MSVCRT:tncleanup.obj
 0001:000091b0       ?__scrt_uninitialize_type_info@@YAXXZ 000000018000a1b0 f   MSVCRT:tncleanup.obj
 0001:000091bc       __local_stdio_printf_options 000000018000a1bc f i MSVCRT:default_local_stdio_options.obj
 0001:000091c4       __local_stdio_scanf_options 000000018000a1c4 f i MSVCRT:default_local_stdio_options.obj
 0001:000091cc       __scrt_initialize_default_local_stdio_options 000000018000a1cc f   MSVCRT:default_local_stdio_options.obj
 0001:000091e8       __scrt_acquire_startup_lock 000000018000a1e8 f   MSVCRT:utility.obj
 0001:00009224       __scrt_dllmain_after_initialize_c 000000018000a224 f   MSVCRT:utility.obj
 0001:00009258       __scrt_dllmain_before_initialize_c 000000018000a258 f   MSVCRT:utility.obj
 0001:00009270       __scrt_dllmain_crt_thread_attach 000000018000a270 f   MSVCRT:utility.obj
 0001:00009298       __scrt_dllmain_crt_thread_detach 000000018000a298 f   MSVCRT:utility.obj
 0001:000092b0       __scrt_dllmain_exception_filter 000000018000a2b0 f   MSVCRT:utility.obj
 0001:00009310       __scrt_dllmain_uninitialize_c 000000018000a310 f   MSVCRT:utility.obj
 0001:00009340       __scrt_dllmain_uninitialize_critical 000000018000a340 f   MSVCRT:utility.obj
 0001:00009354       __scrt_initialize_crt      000000018000a354 f   MSVCRT:utility.obj
 0001:000093a0       __scrt_initialize_onexit_tables 000000018000a3a0 f   MSVCRT:utility.obj
 0001:0000942c       __scrt_is_nonwritable_in_current_image 000000018000a42c f   MSVCRT:utility.obj
 0001:000094c4       __scrt_release_startup_lock 000000018000a4c4 f   MSVCRT:utility.obj
 0001:000094e8       __scrt_uninitialize_crt    000000018000a4e8 f   MSVCRT:utility.obj
 0001:00009514       __scrt_get_dyn_tls_init_callback 000000018000a514 f   MSVCRT:dyn_tls_init.obj
 0001:0000951c       __crt_debugger_hook        000000018000a51c f   MSVCRT:utility_desktop.obj
 0001:00009524       __scrt_fastfail            000000018000a524 f   MSVCRT:utility_desktop.obj
 0001:00009670       _RTC_Initialize            000000018000a670 f   MSVCRT:initsect.obj
 0001:000096ac       _RTC_Terminate             000000018000a6ac f   MSVCRT:initsect.obj
 0001:000096e8       __isa_available_init       000000018000a6e8 f   MSVCRT:cpu_disp.obj
 0001:00009894       __scrt_is_ucrt_dll_in_use  000000018000a894 f   MSVCRT:ucrt_detection.obj
 0001:000098a0       memset                     000000018000a8a0 f   vcruntime:VCRUNTIME140.dll
 0001:000098a6       __C_specific_handler       000000018000a8a6 f   vcruntime:VCRUNTIME140.dll
 0001:000098ac       __std_type_info_destroy_list 000000018000a8ac f   vcruntime:VCRUNTIME140.dll
 0001:000098b2       strlen                     000000018000a8b2 f   ucrt:api-ms-win-crt-string-l1-1-0.dll
 0001:000098b8       _initterm                  000000018000a8b8 f   ucrt:api-ms-win-crt-runtime-l1-1-0.dll
 0001:000098be       _initterm_e                000000018000a8be f   ucrt:api-ms-win-crt-runtime-l1-1-0.dll
 0001:000098c4       _seh_filter_dll            000000018000a8c4 f   ucrt:api-ms-win-crt-runtime-l1-1-0.dll
 0001:000098ca       _configure_narrow_argv     000000018000a8ca f   ucrt:api-ms-win-crt-runtime-l1-1-0.dll
 0001:000098d0       _initialize_narrow_environment 000000018000a8d0 f   ucrt:api-ms-win-crt-runtime-l1-1-0.dll
 0001:000098d6       _initialize_onexit_table   000000018000a8d6 f   ucrt:api-ms-win-crt-runtime-l1-1-0.dll
 0001:000098dc       _execute_onexit_table      000000018000a8dc f   ucrt:api-ms-win-crt-runtime-l1-1-0.dll
 0001:000098e2       _cexit                     000000018000a8e2 f   ucrt:api-ms-win-crt-runtime-l1-1-0.dll
 0001:000098e8       memcpy                     000000018000a8e8 f   vcruntime:VCRUNTIME140.dll
 0001:00009900       _guard_dispatch_icall_nop  000000018000a900 f   MSVCRT:guard_dispatch.obj
 0001:00009920       _guard_xfg_dispatch_icall_nop 000000018000a920 f   MSVCRT:guard_xfg_dispatch.obj
 0002:00000000       __imp_OpenThreadToken      000000018000b000     advapi32:ADVAPI32.dll
 0002:00000008       __imp_ConvertStringSidToSidW 000000018000b008     advapi32:ADVAPI32.dll
 0002:00000010       __imp_ConvertSidToStringSidW 000000018000b010     advapi32:ADVAPI32.dll
 0002:00000018       __imp_LookupPrivilegeValueW 000000018000b018     advapi32:ADVAPI32.dll
 0002:00000020       __imp_LookupAccountNameW   000000018000b020     advapi32:ADVAPI32.dll
 0002:00000028       __imp_LookupAccountSidW    000000018000b028     advapi32:ADVAPI32.dll
 0002:00000030       __imp_SetSecurityDescriptorOwner 000000018000b030     advapi32:ADVAPI32.dll
 0002:00000038       __imp_SetSecurityDescriptorDacl 000000018000b038     advapi32:ADVAPI32.dll
 0002:00000040       __imp_SetFileSecurityW     000000018000b040     advapi32:ADVAPI32.dll
 0002:00000048       __imp_MapGenericMask       000000018000b048     advapi32:ADVAPI32.dll
 0002:00000050       __imp_InitializeSecurityDescriptor 000000018000b050     advapi32:ADVAPI32.dll
 0002:00000058       __imp_InitializeAcl        000000018000b058     advapi32:ADVAPI32.dll
 0002:00000060       __imp_GetTokenInformation  000000018000b060     advapi32:ADVAPI32.dll
 0002:00000068       __imp_GetSecurityDescriptorOwner 000000018000b068     advapi32:ADVAPI32.dll
 0002:00000070       __imp_GetSecurityDescriptorDacl 000000018000b070     advapi32:ADVAPI32.dll
 0002:00000078       __imp_GetLengthSid         000000018000b078     advapi32:ADVAPI32.dll
 0002:00000080       __imp_GetFileSecurityW     000000018000b080     advapi32:ADVAPI32.dll
 0002:00000088       __imp_GetAclInformation    000000018000b088     advapi32:ADVAPI32.dll
 0002:00000090       __imp_GetAce               000000018000b090     advapi32:ADVAPI32.dll
 0002:00000098       __imp_DuplicateTokenEx     000000018000b098     advapi32:ADVAPI32.dll
 0002:000000a0       __imp_RegCloseKey          000000018000b0a0     advapi32:ADVAPI32.dll
 0002:000000a8       __imp_RegOpenKeyExW        000000018000b0a8     advapi32:ADVAPI32.dll
 0002:000000b0       __imp_RegQueryValueExW     000000018000b0b0     advapi32:ADVAPI32.dll
 0002:000000b8       __imp_SetThreadToken       000000018000b0b8     advapi32:ADVAPI32.dll
 0002:000000c0       __imp_OpenProcessToken     000000018000b0c0     advapi32:ADVAPI32.dll
 0002:000000c8       __imp_AddAccessDeniedAceEx 000000018000b0c8     advapi32:ADVAPI32.dll
 0002:000000d0       __imp_AccessCheck          000000018000b0d0     advapi32:ADVAPI32.dll
 0002:000000d8       __imp_AddAccessAllowedAceEx 000000018000b0d8     advapi32:ADVAPI32.dll
 0002:000000e0       __imp_AdjustTokenPrivileges 000000018000b0e0     advapi32:ADVAPI32.dll
 0002:000000e8       \177ADVAPI32_NULL_THUNK_DATA 000000018000b0e8     advapi32:ADVAPI32.dll
 0002:000000f0       __imp_RtlVirtualUnwind     000000018000b0f0     kernel32:KERNEL32.dll
 0002:000000f8       __imp_UnhandledExceptionFilter 000000018000b0f8     kernel32:KERNEL32.dll
 0002:00000100       __imp_SetUnhandledExceptionFilter 000000018000b100     kernel32:KERNEL32.dll
 0002:00000108       __imp_TerminateProcess     000000018000b108     kernel32:KERNEL32.dll
 0002:00000110       __imp_IsProcessorFeaturePresent 000000018000b110     kernel32:KERNEL32.dll
 0002:00000118       __imp_QueryPerformanceCounter 000000018000b118     kernel32:KERNEL32.dll
 0002:00000120       __imp_GetCurrentProcessId  000000018000b120     kernel32:KERNEL32.dll
 0002:00000128       __imp_GetCurrentThreadId   000000018000b128     kernel32:KERNEL32.dll
 0002:00000130       __imp_GetSystemTimeAsFileTime 000000018000b130     kernel32:KERNEL32.dll
 0002:00000138       __imp_DisableThreadLibraryCalls 000000018000b138     kernel32:KERNEL32.dll
 0002:00000140       __imp_InitializeSListHead  000000018000b140     kernel32:KERNEL32.dll
 0002:00000148       __imp_IsDebuggerPresent    000000018000b148     kernel32:KERNEL32.dll
 0002:00000150       __imp_GetVolumeInformationW 000000018000b150     kernel32:KERNEL32.dll
 0002:00000158       __imp_GetVolumePathNameW   000000018000b158     kernel32:KERNEL32.dll
 0002:00000160       __imp_RemoveDirectoryW     000000018000b160     kernel32:KERNEL32.dll
 0002:00000168       __imp_SetEndOfFile         000000018000b168     kernel32:KERNEL32.dll
 0002:00000170       __imp_SetFileAttributesW   000000018000b170     kernel32:KERNEL32.dll
 0002:00000178       __imp_SetFileTime          000000018000b178     kernel32:KERNEL32.dll
 0002:00000180       __imp_UnmapViewOfFile      000000018000b180     kernel32:KERNEL32.dll
 0002:00000188       __imp_GetLogicalDrives     000000018000b188     kernel32:KERNEL32.dll
 0002:00000190       __imp_GetFullPathNameW     000000018000b190     kernel32:KERNEL32.dll
 0002:00000198       __imp_RtlLookupFunctionEntry 000000018000b198     kernel32:KERNEL32.dll
 0002:000001a0       __imp_RtlCaptureContext    000000018000b1a0     kernel32:KERNEL32.dll
 0002:000001a8       __imp_SetFileCompletionNotificationModes 000000018000b1a8     kernel32:KERNEL32.dll
 0002:000001b0       __imp_GetTickCount64       000000018000b1b0     kernel32:KERNEL32.dll
 0002:000001b8       __imp_InitOnceExecuteOnce  000000018000b1b8     kernel32:KERNEL32.dll
 0002:000001c0       __imp_DeleteCriticalSection 000000018000b1c0     kernel32:KERNEL32.dll
 0002:000001c8       __imp_LeaveCriticalSection 000000018000b1c8     kernel32:KERNEL32.dll
 0002:000001d0       __imp_EnterCriticalSection 000000018000b1d0     kernel32:KERNEL32.dll
 0002:000001d8       __imp_InitializeCriticalSection 000000018000b1d8     kernel32:KERNEL32.dll
 0002:000001e0       __imp_AcquireSRWLockShared 000000018000b1e0     kernel32:KERNEL32.dll
 0002:000001e8       __imp_AcquireSRWLockExclusive 000000018000b1e8     kernel32:KERNEL32.dll
 0002:000001f0       __imp_ReleaseSRWLockShared 000000018000b1f0     kernel32:KERNEL32.dll
 0002:000001f8       __imp_ReleaseSRWLockExclusive 000000018000b1f8     kernel32:KERNEL32.dll
 0002:00000200       __imp_InitializeSRWLock    000000018000b200     kernel32:KERNEL32.dll
 0002:00000208       __imp_GetQueuedCompletionStatusEx 000000018000b208     kernel32:KERNEL32.dll
 0002:00000210       __imp_SetLastError         000000018000b210     kernel32:KERNEL32.dll
 0002:00000218       __imp_GetHandleInformation 000000018000b218     kernel32:KERNEL32.dll
 0002:00000220       __imp_CreateSymbolicLinkW  000000018000b220     kernel32:KERNEL32.dll
 0002:00000228       __imp_ReadDirectoryChangesW 000000018000b228     kernel32:KERNEL32.dll
 0002:00000230       __imp_CreateHardLinkW      000000018000b230     kernel32:KERNEL32.dll
 0002:00000238       __imp_MoveFileExW          000000018000b238     kernel32:KERNEL32.dll
 0002:00000240       __imp_CopyFileExW          000000018000b240     kernel32:KERNEL32.dll
 0002:00000248       __imp_LocalFree            000000018000b248     kernel32:KERNEL32.dll
 0002:00000250       __imp_LocalAlloc           000000018000b250     kernel32:KERNEL32.dll
 0002:00000258       __imp_GetProcAddress       000000018000b258     kernel32:KERNEL32.dll
 0002:00000260       __imp_GetModuleHandleW     000000018000b260     kernel32:KERNEL32.dll
 0002:00000268       __imp_GetCurrentThread     000000018000b268     kernel32:KERNEL32.dll
 0002:00000270       __imp_CreateEventW         000000018000b270     kernel32:KERNEL32.dll
 0002:00000278       __imp_CancelIo             000000018000b278     kernel32:KERNEL32.dll
 0002:00000280       __imp_FindNextStreamW      000000018000b280     kernel32:KERNEL32.dll
 0002:00000288       __imp_FlushFileBuffers     000000018000b288     kernel32:KERNEL32.dll
 0002:00000290       __imp_GetDiskFreeSpaceW    000000018000b290     kernel32:KERNEL32.dll
 0002:00000298       __imp_GetFileInformationByHandle 000000018000b298     kernel32:KERNEL32.dll
 0002:000002a0       __imp_GetFileSizeEx        000000018000b2a0     kernel32:KERNEL32.dll
 0002:000002a8       __imp_GetFileType          000000018000b2a8     kernel32:KERNEL32.dll
 0002:000002b0       __imp_LockFileEx           000000018000b2b0     kernel32:KERNEL32.dll
 0002:000002b8       __imp_ReadFile             000000018000b2b8     kernel32:KERNEL32.dll
 0002:000002c0       __imp_SetFileInformationByHandle 000000018000b2c0     kernel32:KERNEL32.dll
 0002:000002c8       __imp_SetFilePointerEx     000000018000b2c8     kernel32:KERNEL32.dll
 0002:000002d0       __imp_UnlockFileEx         000000018000b2d0     kernel32:KERNEL32.dll
 0002:000002d8       __imp_WriteFile            000000018000b2d8     kernel32:KERNEL32.dll
 0002:000002e0       __imp_CloseHandle          000000018000b2e0     kernel32:KERNEL32.dll
 0002:000002e8       __imp_DuplicateHandle      000000018000b2e8     kernel32:KERNEL32.dll
 0002:000002f0       __imp_GetLastError         000000018000b2f0     kernel32:KERNEL32.dll
 0002:000002f8       __imp_DeviceIoControl      000000018000b2f8     kernel32:KERNEL32.dll
 0002:00000300       __imp_GetOverlappedResult  000000018000b300     kernel32:KERNEL32.dll
 0002:00000308       __imp_GetCurrentProcess    000000018000b308     kernel32:KERNEL32.dll
 0002:00000310       __imp_GetSystemInfo        000000018000b310     kernel32:KERNEL32.dll
 0002:00000318       __imp_MapViewOfFile        000000018000b318     kernel32:KERNEL32.dll
 0002:00000320       __imp_GetFinalPathNameByHandleW 000000018000b320     kernel32:KERNEL32.dll
 0002:00000328       __imp_CreateFileMappingA   000000018000b328     kernel32:KERNEL32.dll
 0002:00000330       __imp_ReOpenFile           000000018000b330     kernel32:KERNEL32.dll
 0002:00000338       __imp_CreateIoCompletionPort 000000018000b338     kernel32:KERNEL32.dll
 0002:00000340       __imp_GetQueuedCompletionStatus 000000018000b340     kernel32:KERNEL32.dll
 0002:00000348       __imp_PostQueuedCompletionStatus 000000018000b348     kernel32:KERNEL32.dll
 0002:00000350       __imp_FormatMessageW       000000018000b350     kernel32:KERNEL32.dll
 0002:00000358       __imp_FlushViewOfFile      000000018000b358     kernel32:KERNEL32.dll
 0002:00000360       __imp_SetHandleInformation 000000018000b360     kernel32:KERNEL32.dll
 0002:00000368       __imp_CreateDirectoryW     000000018000b368     kernel32:KERNEL32.dll
 0002:00000370       __imp_CreateFileW          000000018000b370     kernel32:KERNEL32.dll
 0002:00000378       __imp_DeleteFileW          000000018000b378     kernel32:KERNEL32.dll
 0002:00000380       __imp_FindClose            000000018000b380     kernel32:KERNEL32.dll
 0002:00000388       __imp_FindFirstFileW       000000018000b388     kernel32:KERNEL32.dll
 0002:00000390       __imp_FindNextFileW        000000018000b390     kernel32:KERNEL32.dll
 0002:00000398       __imp_GetDiskFreeSpaceExW  000000018000b398     kernel32:KERNEL32.dll
 0002:000003a0       __imp_GetDriveTypeW        000000018000b3a0     kernel32:KERNEL32.dll
 0002:000003a8       __imp_GetFileAttributesW   000000018000b3a8     kernel32:KERNEL32.dll
 0002:000003b0       __imp_GetFileAttributesExW 000000018000b3b0     kernel32:KERNEL32.dll
 0002:000003b8       __imp_FindFirstStreamW     000000018000b3b8     kernel32:KERNEL32.dll
 0002:000003c0       \177KERNEL32_NULL_THUNK_DATA 000000018000b3c0     kernel32:KERNEL32.dll
 0002:000003c8       __imp_TransmitFile         000000018000b3c8     mswsock:MSWSOCK.dll
 0002:000003d0       \177MSWSOCK_NULL_THUNK_DATA 000000018000b3d0     mswsock:MSWSOCK.dll
 0002:000003d8       __imp_memset               000000018000b3d8     vcruntime:VCRUNTIME140.dll
 0002:000003e0       __imp___C_specific_handler 000000018000b3e0     vcruntime:VCRUNTIME140.dll
 0002:000003e8       __imp___std_type_info_destroy_list 000000018000b3e8     vcruntime:VCRUNTIME140.dll
 0002:000003f0       __imp_memcpy               000000018000b3f0     vcruntime:VCRUNTIME140.dll
 0002:000003f8       \177VCRUNTIME140_NULL_THUNK_DATA 000000018000b3f8     vcruntime:VCRUNTIME140.dll
 0002:00000400       __imp_WSAStartup           000000018000b400     ws2_32:WS2_32.dll
 0002:00000408       __imp_WSASocketW           000000018000b408     ws2_32:WS2_32.dll
 0002:00000410       __imp_WSAEnumProtocolsW    000000018000b410     ws2_32:WS2_32.dll
 0002:00000418       __imp_bind                 000000018000b418     ws2_32:WS2_32.dll
 0002:00000420       __imp_closesocket          000000018000b420     ws2_32:WS2_32.dll
 0002:00000428       __imp_inet_ntop            000000018000b428     ws2_32:WS2_32.dll
 0002:00000430       __imp_socket               000000018000b430     ws2_32:WS2_32.dll
 0002:00000438       __imp_shutdown             000000018000b438     ws2_32:WS2_32.dll
 0002:00000440       __imp_setsockopt           000000018000b440     ws2_32:WS2_32.dll
 0002:00000448       __imp_ntohl                000000018000b448     ws2_32:WS2_32.dll
 0002:00000450       __imp_listen               000000018000b450     ws2_32:WS2_32.dll
 0002:00000458       __imp_htonl                000000018000b458     ws2_32:WS2_32.dll
 0002:00000460       __imp_getsockopt           000000018000b460     ws2_32:WS2_32.dll
 0002:00000468       __imp_getsockname          000000018000b468     ws2_32:WS2_32.dll
 0002:00000470       __imp_getpeername          000000018000b470     ws2_32:WS2_32.dll
 0002:00000478       __imp_accept               000000018000b478     ws2_32:WS2_32.dll
 0002:00000480       __imp___WSAFDIsSet         000000018000b480     ws2_32:WS2_32.dll
 0002:00000488       __imp_WSAEventSelect       000000018000b488     ws2_32:WS2_32.dll
 0002:00000490       __imp_send                 000000018000b490     ws2_32:WS2_32.dll
 0002:00000498       __imp_recv                 000000018000b498     ws2_32:WS2_32.dll
 0002:000004a0       __imp_ioctlsocket          000000018000b4a0     ws2_32:WS2_32.dll
 0002:000004a8       __imp_WSASend              000000018000b4a8     ws2_32:WS2_32.dll
 0002:000004b0       __imp_WSARecv              000000018000b4b0     ws2_32:WS2_32.dll
 0002:000004b8       __imp_WSAIoctl             000000018000b4b8     ws2_32:WS2_32.dll
 0002:000004c0       __imp_WSAGetLastError      000000018000b4c0     ws2_32:WS2_32.dll
 0002:000004c8       __imp_sendto               000000018000b4c8     ws2_32:WS2_32.dll
 0002:000004d0       __imp_select               000000018000b4d0     ws2_32:WS2_32.dll
 0002:000004d8       __imp_recvfrom             000000018000b4d8     ws2_32:WS2_32.dll
 0002:000004e0       __imp_connect              000000018000b4e0     ws2_32:WS2_32.dll
 0002:000004e8       \177WS2_32_NULL_THUNK_DATA 000000018000b4e8     ws2_32:WS2_32.dll
 0002:000004f0       __imp_malloc               000000018000b4f0     ucrt:api-ms-win-crt-heap-l1-1-0.dll
 0002:000004f8       __imp_free                 000000018000b4f8     ucrt:api-ms-win-crt-heap-l1-1-0.dll
 0002:00000500       \177api-ms-win-crt-heap-l1-1-0_NULL_THUNK_DATA 000000018000b500     ucrt:api-ms-win-crt-heap-l1-1-0.dll
 0002:00000508       __imp__initterm            000000018000b508     ucrt:api-ms-win-crt-runtime-l1-1-0.dll
 0002:00000510       __imp__cexit               000000018000b510     ucrt:api-ms-win-crt-runtime-l1-1-0.dll
 0002:00000518       __imp__initialize_onexit_table 000000018000b518     ucrt:api-ms-win-crt-runtime-l1-1-0.dll
 0002:00000520       __imp__initialize_narrow_environment 000000018000b520     ucrt:api-ms-win-crt-runtime-l1-1-0.dll
 0002:00000528       __imp__configure_narrow_argv 000000018000b528     ucrt:api-ms-win-crt-runtime-l1-1-0.dll
 0002:00000530       __imp_abort                000000018000b530     ucrt:api-ms-win-crt-runtime-l1-1-0.dll
 0002:00000538       __imp__errno               000000018000b538     ucrt:api-ms-win-crt-runtime-l1-1-0.dll
 0002:00000540       __imp__initterm_e          000000018000b540     ucrt:api-ms-win-crt-runtime-l1-1-0.dll
 0002:00000548       __imp__execute_onexit_table 000000018000b548     ucrt:api-ms-win-crt-runtime-l1-1-0.dll
 0002:00000550       __imp__seh_filter_dll      000000018000b550     ucrt:api-ms-win-crt-runtime-l1-1-0.dll
 0002:00000558       \177api-ms-win-crt-runtime-l1-1-0_NULL_THUNK_DATA 000000018000b558     ucrt:api-ms-win-crt-runtime-l1-1-0.dll
 0002:00000560       __imp_strncpy              000000018000b560     ucrt:api-ms-win-crt-string-l1-1-0.dll
 0002:00000568       __imp_strlen               000000018000b568     ucrt:api-ms-win-crt-string-l1-1-0.dll
 0002:00000570       __imp_wcslen               000000018000b570     ucrt:api-ms-win-crt-string-l1-1-0.dll
 0002:00000578       \177api-ms-win-crt-string-l1-1-0_NULL_THUNK_DATA 000000018000b578     ucrt:api-ms-win-crt-string-l1-1-0.dll
 0002:00000580       __imp_JNU_ThrowIOExceptionWithLastError 000000018000b580     java:java.dll
 0002:00000588       __imp_Java_sun_security_provider_NativeSeedGenerator_nativeGenerateSeed 000000018000b588     java:java.dll
 0002:00000590       __imp_JNU_NewObjectByName  000000018000b590     java:java.dll
 0002:00000598       __imp_JNU_ThrowByName      000000018000b598     java:java.dll
 0002:000005a0       __imp_JNU_ThrowInternalError 000000018000b5a0     java:java.dll
 0002:000005a8       __imp_JNU_ThrowOutOfMemoryError 000000018000b5a8     java:java.dll
 0002:000005b0       __imp_JNU_ThrowIOException 000000018000b5b0     java:java.dll
 0002:000005b8       \177java_NULL_THUNK_DATA   000000018000b5b8     java:java.dll
 0002:000005c0       __imp_NET_ThrowNew         000000018000b5c0     net:net.dll
 0002:000005c8       __imp_NET_WinBind          000000018000b5c8     net:net.dll
 0002:000005d0       __imp_NET_EnableFastTcpLoopbackConnect 000000018000b5d0     net:net.dll
 0002:000005d8       __imp_initInetAddressIDs   000000018000b5d8     net:net.dll
 0002:000005e0       __imp_ipv6_available       000000018000b5e0     net:net.dll
 0002:000005e8       __imp_NET_SockaddrToInetAddress 000000018000b5e8     net:net.dll
 0002:000005f0       __imp_NET_GetPortFromSockaddr 000000018000b5f0     net:net.dll
 0002:000005f8       __imp_NET_GetSockOpt       000000018000b5f8     net:net.dll
 0002:00000600       __imp_NET_SetSockOpt       000000018000b600     net:net.dll
 0002:00000608       __imp_NET_EnableFastTcpLoopback 000000018000b608     net:net.dll
 0002:00000610       __imp_NET_InetAddressToSockaddr 000000018000b610     net:net.dll
 0002:00000618       \177net_NULL_THUNK_DATA    000000018000b618     net:net.dll
 0002:00000620       __guard_check_icall_fptr   000000018000b620     MSVCRT:guard_support.obj
 0002:00000628       __guard_xfg_check_icall_fptr 000000018000b628     MSVCRT:guard_support.obj
 0002:00000630       __guard_dispatch_icall_fptr 000000018000b630     MSVCRT:guard_support.obj
 0002:00000638       __guard_xfg_dispatch_icall_fptr 000000018000b638     MSVCRT:guard_support.obj
 0002:00000640       __guard_xfg_table_dispatch_icall_fptr 000000018000b640     MSVCRT:guard_support.obj
 0002:00000648       __castguard_check_failure_os_handled_fptr 000000018000b648     MSVCRT:guard_support.obj
 0002:00000650       __guard_memcpy_fptr        000000018000b650     vcruntime:softmemtag.obj
 0002:00000658       __xc_a                     000000018000b658     MSVCRT:initializers.obj
 0002:00000660       __xc_z                     000000018000b660     MSVCRT:initializers.obj
 0002:00000668       __xi_a                     000000018000b668     MSVCRT:initializers.obj
 0002:00000670       __xi_z                     000000018000b670     MSVCRT:initializers.obj
 0002:00000678       __xp_a                     000000018000b678     MSVCRT:initializers.obj
 0002:00000680       __xp_z                     000000018000b680     MSVCRT:initializers.obj
 0002:00000688       __xt_a                     000000018000b688     MSVCRT:initializers.obj
 0002:00000690       __xt_z                     000000018000b690     MSVCRT:initializers.obj
 0002:000006a0       ??_C@_07KAIBNCHO@connect@  000000018000b6a0     DatagramChannelImpl.obj
 0002:000006a8       ??_C@_0CC@BDDMPFBF@java?1net?1PortUnreachableExcepti@ 000000018000b6a8     DatagramChannelImpl.obj
 0002:000006d0       ??_C@_08HMBBGFHE@recvfrom@ 000000018000b6d0     DatagramChannelImpl.obj
 0002:000006dc       ??_C@_06MEPBGKEC@sendto@   000000018000b6dc     DatagramChannelImpl.obj
 0002:000006e8       ??_C@_0P@DGIIHHAE@WSARecv?5failed@ 000000018000b6e8     DatagramDispatcher.obj
 0002:000006f8       ??_C@_0P@NKOFNKCM@WSASend?5failed@ 000000018000b6f8     DatagramDispatcher.obj
 0002:00000708       ??_C@_0P@EFDAIKIF@Invalid?5handle@ 000000018000b708     FileDispatcherImpl.obj
 0002:00000718       ??_C@_0M@DCKEEFAG@Read?5failed@ 000000018000b718     FileDispatcherImpl.obj
 0002:00000728       ??_C@_0M@HPFDGGMC@Seek?5failed@ 000000018000b728     FileDispatcherImpl.obj
 0002:00000738       ??_C@_0N@PGCLODBC@Write?5failed@ 000000018000b738     FileDispatcherImpl.obj
 0002:00000748       ??_C@_0BI@ICELLBHO@SetFilePointerEx?5failed@ 000000018000b748     FileDispatcherImpl.obj
 0002:00000760       ??_C@_0N@EFKIKJEB@Force?5failed@ 000000018000b760     FileDispatcherImpl.obj
 0002:00000770       ??_C@_0BC@FODOCFKM@Truncation?5failed@ 000000018000b770     FileDispatcherImpl.obj
 0002:00000788       ??_C@_0M@GLCOPFPC@Size?5failed@ 000000018000b788     FileDispatcherImpl.obj
 0002:00000798       ??_C@_0BB@DDIHOFNN@Available?5failed@ 000000018000b798     FileDispatcherImpl.obj
 0002:000007b0       ??_C@_0P@EMLEKIJM@isOther?5failed@ 000000018000b7b0     FileDispatcherImpl.obj
 0002:000007c0       ??_C@_0M@OOGODMIM@Lock?5failed@ 000000018000b7c0     FileDispatcherImpl.obj
 0002:000007d0       ??_C@_0P@MAMCLOFD@Release?5failed@ 000000018000b7d0     FileDispatcherImpl.obj
 0002:000007e0       ??_C@_0N@GNNFMAIG@Close?5failed@ 000000018000b7e0     FileDispatcherImpl.obj
 0002:000007f0       ??_C@_0BH@OPJFPPPK@DuplicateHandle?5failed@ 000000018000b7f0     FileDispatcherImpl.obj
 0002:00000810       ??_C@_0EC@BGNPHEAP@should?5never?5call?5map?5on?5platfo@ 000000018000b810     FileDispatcherImpl.obj
 0002:00000858       ??_C@_0L@DPMFILPJ@Map?5failed@ 000000018000b858     FileDispatcherImpl.obj
 0002:00000868       ??_C@_0N@IGMMIDE@Unmap?5failed@ 000000018000b868     FileDispatcherImpl.obj
 0002:00000878       ??_C@_0BA@CJMHIODJ@transfer?5failed@ 000000018000b878     FileDispatcherImpl.obj
 0002:00000888       ??_C@_0BG@JDMBHIAK@DirectIO?5setup?5failed@ 000000018000b888     FileDispatcherImpl.obj
 0002:000008a0       ??_C@_0CC@EJDNCKME@GetFileInformationByHandle?5fail@ 000000018000b8a0     FileKey.obj
 0002:000008c8       ??_C@_0BH@MPHCPCAM@java?1io?1FileDescriptor@ 000000018000b8c8     IOUtil.obj
 0002:000008e0       ??_C@_01JPJNBJEM@I@        000000018000b8e0     IOUtil.obj
 0002:000008e4       ??_C@_02ENHFDPNM@fd@       000000018000b8e4     IOUtil.obj
 0002:000008e8       ??_C@_01LELAEKIP@J@        000000018000b8e8     IOUtil.obj
 0002:000008ec       ??_C@_06NCGDPKCC@handle@   000000018000b8ec     IOUtil.obj
 0002:000008f8       ??_C@_0BC@PPBACNOJ@Read?1write?5failed@ 000000018000b8f8     IOUtil.obj
 0002:00000910       ??_C@_0M@PBPOCKDG@ioctlsocket@ 000000018000b910     IOUtil.obj
 0002:00000920       ??_C@_0M@KMFGCEDE@recv?5failed@ 000000018000b920     IOUtil.obj
 0002:00000930       ??_C@_0M@EADLIJBM@send?5failed@ 000000018000b930     IOUtil.obj
 0002:00000940       ??_C@_0CB@EANIAHBH@sun?1nio?1ch?1Iocp$CompletionStatu@ 000000018000b940     Iocp.obj
 0002:00000964       ??_C@_05KKCIMGE@error@     000000018000b964     Iocp.obj
 0002:00000970       ??_C@_0BB@LMCKIICB@bytesTransferred@ 000000018000b970     Iocp.obj
 0002:00000988       ??_C@_0O@HHOLMKBG@completionKey@ 000000018000b988     Iocp.obj
 0002:00000998       ??_C@_0L@GFMJGGB@overlapped@ 000000018000b998     Iocp.obj
 0002:000009a8       ??_C@_0BO@HNKCMKLP@CreateIoCompletionPort?5failed@ 000000018000b9a8     Iocp.obj
 0002:000009c8       ??_C@_0CB@GOEOMHMA@GetQueuedCompletionStatus?5faile@ 000000018000b9c8     Iocp.obj
 0002:000009f0       ??_C@_0BL@IDOBBHMP@PostQueuedCompletionStatus@ 000000018000b9f0     Iocp.obj
 0002:00000a10       ??_C@_09MIBPPDMB@isLoaded0@ 000000018000ba10     MappedMemoryUtils.obj
 0002:00000a1c       ??_C@_06KBCAEOHA@?$CIJJJ?$CJZ@ 000000018000ba1c     MappedMemoryUtils.obj
 0002:00000a24       ??_C@_05DJGLLEII@load0@    000000018000ba24     MappedMemoryUtils.obj
 0002:00000a2c       ??_C@_05JIFFKGAL@?$CIJJ?$CJV@ 000000018000ba2c     MappedMemoryUtils.obj
 0002:00000a38       ??_C@_07NCLCGCAO@unload0@  000000018000ba38     MappedMemoryUtils.obj
 0002:00000a40       ??_C@_06EIIMDAKL@force0@   000000018000ba40     MappedMemoryUtils.obj
 0002:00000a48       ??_C@_0BO@HHHLHKAN@?$CILjava?1io?1FileDescriptor?$DLJJ?$CJV@ 000000018000ba48     MappedMemoryUtils.obj
 0002:00000a68       ??_C@_0N@MNOMAIIN@Flush?5failed@ 000000018000ba68     MappedMemoryUtils.obj
 0002:00000a78       ??_C@_0BL@HBNNAPLM@java?1net?1InetSocketAddress@ 000000018000ba78     Net.obj
 0002:00000a98       ??_C@_0BL@KCCEIBDI@?$CILjava?1net?1InetAddress?$DLI?$CJV@ 000000018000ba98     Net.obj
 0002:00000ab4       ??_C@_06FALKBLGB@?$DMinit?$DO@ 000000018000bab4     Net.obj
 0002:00000abc       ??_C@_06HBELJPBO@socket@   000000018000babc     Net.obj
 0002:00000ac8       ??_C@_0N@JOEJINBO@fastLoopback@ 000000018000bac8     Net.obj
 0002:00000ad8       ??_C@_04NPNJNMMP@bind@     000000018000bad8     Net.obj
 0002:00000ae0       ??_C@_06OODDLKLE@listen@   000000018000bae0     Net.obj
 0002:00000ae8       ??_C@_04LEMNCIAK@?$AI?$PP?$AE?$AE@ 000000018000bae8     Net.obj
 0002:00000af0       ??_C@_05IEANOBDC@?$AI?$PP?$AE?$AE?$AE@ 000000018000baf0     Net.obj
 0002:00000af8       ??_C@_0O@BMGFIIHF@Accept?5failed@ 000000018000baf8     Net.obj
 0002:00000b08       ??_C@_0M@ODFENJLC@getsockname@ 000000018000bb08     Net.obj
 0002:00000b18       ??_C@_0L@DEFCDCGF@getsockopt@ 000000018000bb18     Net.obj
 0002:00000b28       ??_C@_0N@GIECLHOG@setsocketopt@ 000000018000bb28     Net.obj
 0002:00000b38       ??_C@_0L@CKHNIFCM@setsockopt@ 000000018000bb38     Net.obj
 0002:00000b48       ??_C@_0CI@LHHOJOJM@setsocketopt?5to?5block?5or?5unbloc@ 000000018000bb48     Net.obj
 0002:00000b70       ??_C@_08FIACBBDA@shutdown@ 000000018000bb70     Net.obj
 0002:00000b7c       ??_C@_06LGNCCACI@select@   000000018000bb7c     Net.obj
 0002:00000b88       ??_C@_0BB@KKIOKPBC@Connection?5reset@ 000000018000bb88     SocketDispatcher.obj
 0002:00000ba0       ??_C@_0CB@LJKAIJOC@sun?1net?1ConnectionResetExceptio@ 000000018000bba0     SocketDispatcher.obj
 0002:00000bc8       ??_C@_0BD@MOAOKNAP@Vector?5read?5failed@ 000000018000bbc8     SocketDispatcher.obj
 0002:00000be0       ??_C@_0BJ@FJAMCHKE@Connection?5reset?5by?5peer@ 000000018000bbe0     SocketDispatcher.obj
 0002:00000c00       ??_C@_0BE@IPALPBFO@Vector?5write?5failed@ 000000018000bc00     SocketDispatcher.obj
 0002:00000c14       ??_C@_01NKEKCIAE@?$AE@     000000018000bc14     SocketDispatcher.obj
 0002:00000c18       ??_C@_0BE@EFPANNNH@Socket?5close?5failed@ 000000018000bc18     SocketDispatcher.obj
 0002:00000c30       ??_C@_0BN@BEOHNNJC@Unix?5domain?5path?5not?5present@ 000000018000bc30     UnixDomainSockets.obj
 0002:00000c50       ??_C@_0BJ@IJNLNPKI@java?1net?1SocketException@ 000000018000bc50     UnixDomainSockets.obj
 0002:00000c70       ??_C@_0BK@HNBAHHNO@Unix?5domain?5path?5too?5long@ 000000018000bc70     UnixDomainSockets.obj
 0002:00000c90       ??_C@_0L@DCBIFDBE@WSASocketW@ 000000018000bc90     UnixDomainSockets.obj
 0002:00000c9c       ??_C@_03ILCNEGFN@?$AE?$PP?$AE@ 000000018000bc9c     UnixDomainSockets.obj
 0002:00000ca0       ??_C@_0BF@CMKNLFPM@epoll_create1?5failed@ 000000018000bca0     WEPollNatives.obj
 0002:00000cb8       ??_C@_0BC@POABAMPF@epoll_wait?5failed@ 000000018000bcb8     WEPollNatives.obj
 0002:00000cd0       ??_C@_0BA@KDJDNLHD@ReadFile?5failed@ 000000018000bcd0     WindowsAsynchronousFileChannelImpl.obj
 0002:00000ce0       ??_C@_0BB@IBAPLIEE@WriteFile?5failed@ 000000018000bce0     WindowsAsynchronousFileChannelImpl.obj
 0002:00000cf8       ??_C@_0BA@MECHHPMI@LockFile?5failed@ 000000018000bcf8     WindowsAsynchronousFileChannelImpl.obj
 0002:00000d08       ??_C@_0O@FPJGNADN@socket?5failed@ 000000018000bd08     WindowsAsynchronousServerSocketChannelImpl.obj
 0002:00000d18       ??_C@_0BA@PBEMOOLP@WSAIoctl?5failed@ 000000018000bd18     WindowsAsynchronousServerSocketChannelImpl.obj
 0002:00000d28       ??_C@_0BA@CMPAPNB@AcceptEx?5failed@ 000000018000bd28     WindowsAsynchronousServerSocketChannelImpl.obj
 0002:00000d38       ??_C@_0BC@PAEKIADO@setsockopt?5failed@ 000000018000bd38     WindowsAsynchronousServerSocketChannelImpl.obj
 0002:00000d50       ??_C@_0BD@FFLNFFAC@closesocket?5failed@ 000000018000bd50     WindowsAsynchronousServerSocketChannelImpl.obj
 0002:00000d68       ??_C@_0BB@COIIDLME@ConnectEx?5failed@ 000000018000bd68     WindowsAsynchronousSocketChannelImpl.obj
 0002:00000d80       ??_C@_0BA@GMHHDNNI@shutdown?5failed@ 000000018000bd80     WindowsAsynchronousSocketChannelImpl.obj
 0002:00000d90       ??_C@_04PFANPMCN@?$CII?$CJV@ 000000018000bd90     WindowsNativeDispatcher.obj
 0002:00000d98       ??_C@_0BM@FOMEEEOI@sun?1nio?1fs?1WindowsException@ 000000018000bd98     WindowsNativeDispatcher.obj
 0002:00000db8       ??_C@_0CN@IAHHKCCP@sun?1nio?1fs?1WindowsNativeDispatc@ 000000018000bdb8     WindowsNativeDispatcher.obj
 0002:00000de8       ??_C@_0BD@JFADHEFE@Ljava?1lang?1String?$DL@ 000000018000bde8     WindowsNativeDispatcher.obj
 0002:00000dfc       ??_C@_04MEMAJGDJ@name@     000000018000bdfc     WindowsNativeDispatcher.obj
 0002:00000e08       ??_C@_0L@HNMJPKNA@attributes@ 000000018000be08     WindowsNativeDispatcher.obj
 0002:00000e18       ??_C@_0CP@OGPMEFOM@sun?1nio?1fs?1WindowsNativeDispatc@ 000000018000be18     WindowsNativeDispatcher.obj
 0002:00000e48       ??_C@_0DF@OBLOOIFM@sun?1nio?1fs?1WindowsNativeDispatc@ 000000018000be48     WindowsNativeDispatcher.obj
 0002:00000e80       ??_C@_0P@BFNHNOMJ@fileSystemName@ 000000018000be80     WindowsNativeDispatcher.obj
 0002:00000e90       ??_C@_0L@HCGAGGAJ@volumeName@ 000000018000be90     WindowsNativeDispatcher.obj
 0002:00000ea0       ??_C@_0BD@ILMPNPNH@volumeSerialNumber@ 000000018000bea0     WindowsNativeDispatcher.obj
 0002:00000eb4       ??_C@_05GECEPKB@flags@     000000018000beb4     WindowsNativeDispatcher.obj
 0002:00000ec0       ??_C@_0DB@OGAJBKPO@sun?1nio?1fs?1WindowsNativeDispatc@ 000000018000bec0     WindowsNativeDispatcher.obj
 0002:00000ef8       ??_C@_0BD@LDNCHAFG@freeBytesAvailable@ 000000018000bef8     WindowsNativeDispatcher.obj
 0002:00000f10       ??_C@_0BD@FIEGHADN@totalNumberOfBytes@ 000000018000bf10     WindowsNativeDispatcher.obj
 0002:00000f28       ??_C@_0BH@DLDLDEPI@totalNumberOfFreeBytes@ 000000018000bf28     WindowsNativeDispatcher.obj
 0002:00000f40       ??_C@_0P@EEANGJCF@bytesPerSector@ 000000018000bf40     WindowsNativeDispatcher.obj
 0002:00000f50       ??_C@_0CL@IEKIAJIE@sun?1nio?1fs?1WindowsNativeDispatc@ 000000018000bf50     WindowsNativeDispatcher.obj
 0002:00000f7c       ??_C@_06LKIIGAOE@domain@   000000018000bf7c     WindowsNativeDispatcher.obj
 0002:00000f84       ??_C@_03MMGHDJKG@use@      000000018000bf84     WindowsNativeDispatcher.obj
 0002:00000f88       ??_C@_0DC@CMOGENGN@sun?1nio?1fs?1WindowsNativeDispatc@ 000000018000bf88     WindowsNativeDispatcher.obj
 0002:00000fc0       ??_C@_08BCFBCIIE@aceCount@ 000000018000bfc0     WindowsNativeDispatcher.obj
 0002:00000fd0       ??_C@_0DE@MGDINMHA@sun?1nio?1fs?1WindowsNativeDispatc@ 000000018000bfd0     WindowsNativeDispatcher.obj
 0002:00001008       ??_C@_1BK@MGMFAEKH@?$AAk?$AAe?$AAr?$AAn?$AAe?$AAl?$AA3?$AA2?$AA?4?$AAd?$AAl?$AAl@ 000000018000c008     WindowsNativeDispatcher.obj
 0002:00001028       ??_C@_0BJ@IGDICJAB@GetFileInformationByName@ 000000018000c028     WindowsNativeDispatcher.obj
 0002:00001048       ??_C@_0BG@PMFIMNNM@should?5not?5reach?5here@ 000000018000c048     WindowsNativeDispatcher.obj
 0002:00001060       ??_C@_0CC@NMODGIKH@Unable?5to?5allocate?5LUID?5structu@ 000000018000c060     WindowsNativeDispatcher.obj
 0002:00001088       ??_C@_0BI@COMCEALI@GetFullPathNameW?5failed@ 000000018000c088     WindowsNativeDispatcher.obj
 0002:000010a0       ??_C@_0CB@DJOGFDBC@native?5memory?5allocation?5failur@ 000000018000c0a0     WindowsNativeDispatcher.obj
 0002:000010c8       ??_C@_0CB@BLMDNHEM@GetFinalPathNameByHandleW?5faile@ 000000018000c0c8     WindowsNativeDispatcher.obj
 0002:000010f0       ??_C@_0O@IFFBAKPD@Select?5failed@ 000000018000c0f0     WindowsSelectorImpl.obj
 0002:00001100       ??_C@_05GCIPIGEI@Debug@    000000018000c100     nio_util.obj
 0002:00001108       ??_C@_09FBNMMHMJ@Exception@ 000000018000c108     nio_util.obj
 0002:00001114       ??_C@_05GCNIINAF@Event@    000000018000c114     nio_util.obj
 0002:0000111c       ??_C@_04LBABLPF@Exit@      000000018000c11c     nio_util.obj
 0002:00001124       ??_C@_05HKHPEFOF@Entry@    000000018000c124     nio_util.obj
 0002:00001130       ??_C@_07NKEHFKFB@jcl_nio@  000000018000c130     nio_util.obj
 0002:00001138       ??_C@_0BC@DGCLLADE@J9TraceFormat?4dat@ 000000018000c138     nio_util.obj
 0002:00001150       ??_C@_1CG@MIHFGBDO@?$AA?2?$AAD?$AAe?$AAv?$AAi?$AAc?$AAe?$AA?2?$AAA?$AAf?$AAd?$AA?2?$AAW?$AAe?$AAp@ 000000018000c150     wepoll.obj
 0002:00001178       ??_C@_1BE@GJOFHIHD@?$AAn?$AAt?$AAd?$AAl?$AAl?$AA?4?$AAd?$AAl?$AAl@ 000000018000c178     wepoll.obj
 0002:00001190       ??_C@_0BB@BIKHJNEF@NtCancelIoFileEx@ 000000018000c190     wepoll.obj
 0002:000011a8       ??_C@_0N@KPMLACHP@NtCreateFile@ 000000018000c1a8     wepoll.obj
 0002:000011b8       ??_C@_0BD@JHDPIODG@NtCreateKeyedEvent@ 000000018000c1b8     wepoll.obj
 0002:000011d0       ??_C@_0BG@PCMBHBNE@NtDeviceIoControlFile@ 000000018000c1d0     wepoll.obj
 0002:000011e8       ??_C@_0BE@EHEKCOOF@NtReleaseKeyedEvent@ 000000018000c1e8     wepoll.obj
 0002:00001200       ??_C@_0BE@KJOMDIDG@NtWaitForKeyedEvent@ 000000018000c200     wepoll.obj
 0002:00001218       ??_C@_0BG@NFNCIOML@RtlNtStatusToDosError@ 000000018000c218     wepoll.obj
 0002:00001240       _pDefaultRawDllMain        000000018000c240     MSVCRT:dll_dllmain.obj
 0002:00001240       _pRawDllMain               000000018000c240     MSVCRT:dll_dllmain.obj
 0002:00001250       __xmm@ffffffffffffffffffffffffffffffff 000000018000c250     MSVCRT:utility.obj
 0002:00001260       _load_config_used          000000018000c260     MSVCRT:loadcfg.obj
 0002:00001480       __volatile_metadata        000000018000c480     <linker-defined>
 0002:000017c0       __rtc_iaa                  000000018000c7c0     MSVCRT:initsect.obj
 0002:000017c8       __rtc_izz                  000000018000c7c8     MSVCRT:initsect.obj
 0002:000017d0       __rtc_taa                  000000018000c7d0     MSVCRT:initsect.obj
 0002:000017d8       __rtc_tzz                  000000018000c7d8     MSVCRT:initsect.obj
 0002:00004ebc       __IMPORT_DESCRIPTOR_java   000000018000febc     java:java.dll
 0002:00004ed0       __IMPORT_DESCRIPTOR_net    000000018000fed0     net:net.dll
 0002:00004ee4       __IMPORT_DESCRIPTOR_ADVAPI32 000000018000fee4     advapi32:ADVAPI32.dll
 0002:00004ef8       __IMPORT_DESCRIPTOR_MSWSOCK 000000018000fef8     mswsock:MSWSOCK.dll
 0002:00004f0c       __IMPORT_DESCRIPTOR_WS2_32 000000018000ff0c     ws2_32:WS2_32.dll
 0002:00004f20       __IMPORT_DESCRIPTOR_KERNEL32 000000018000ff20     kernel32:KERNEL32.dll
 0002:00004f34       __IMPORT_DESCRIPTOR_VCRUNTIME140 000000018000ff34     vcruntime:VCRUNTIME140.dll
 0002:00004f48       __IMPORT_DESCRIPTOR_api-ms-win-crt-heap-l1-1-0 000000018000ff48     ucrt:api-ms-win-crt-heap-l1-1-0.dll
 0002:00004f5c       __IMPORT_DESCRIPTOR_api-ms-win-crt-string-l1-1-0 000000018000ff5c     ucrt:api-ms-win-crt-string-l1-1-0.dll
 0002:00004f70       __IMPORT_DESCRIPTOR_api-ms-win-crt-runtime-l1-1-0 000000018000ff70     ucrt:api-ms-win-crt-runtime-l1-1-0.dll
 0002:00004f84       __NULL_IMPORT_DESCRIPTOR   000000018000ff84     java:java.dll
 0003:00000080       jcl_nio_UtModuleInfo       0000000180012080     nio_util.obj
 0003:000000e8       jcl_nio_UtTraceVersionInfo 00000001800120e8     nio_util.obj
 0003:000000ec       jcl_nio_UtLevels           00000001800120ec     nio_util.obj
 0003:000000f8       jcl_nio_group4             00000001800120f8     nio_util.obj
 0003:00000118       jcl_nio_group3             0000000180012118     nio_util.obj
 0003:00000138       jcl_nio_tpids2             0000000180012138     nio_util.obj
 0003:00000150       jcl_nio_group2             0000000180012150     nio_util.obj
 0003:00000170       jcl_nio_group1             0000000180012170     nio_util.obj
 0003:00000190       jcl_nio_group0             0000000180012190     nio_util.obj
 0003:000001f0       __security_cookie          00000001800121f0     MSVCRT:gs_cookie.obj
 0003:000001f8       __security_cookie_complement 00000001800121f8     MSVCRT:gs_cookie.obj
 0003:00000200       __scrt_native_dllmain_reason 0000000180012200     MSVCRT:utility.obj
 0003:00000208       __isa_available            0000000180012208     MSVCRT:cpu_disp.obj
 0003:0000020c       __isa_enabled              000000018001220c     MSVCRT:cpu_disp.obj
 0003:00000210       __memset_fast_string_threshold 0000000180012210     MSVCRT:cpu_disp.obj
 0003:00000218       __memset_nt_threshold      0000000180012218     MSVCRT:cpu_disp.obj
 0003:00000220       __scrt_ucrt_dll_is_in_use  0000000180012220     MSVCRT:ucrt_stubs.obj
 0003:000005b8       jcl_nio_UtActive           00000001800125b8     nio_util.obj
 0003:00000ba0       ?__type_info_root_node@@3U__type_info_node@@A 0000000180012ba0     MSVCRT:tncleanup.obj
 0003:00000bb0       ?_OptionsStorage@?1??__local_stdio_printf_options@@9@4_KA 0000000180012bb0     MSVCRT:default_local_stdio_options.obj
 0003:00000bb8       ?_OptionsStorage@?1??__local_stdio_scanf_options@@9@4_KA 0000000180012bb8     MSVCRT:default_local_stdio_options.obj
 0003:00000bc0       __scrt_current_native_startup_state 0000000180012bc0     MSVCRT:utility.obj
 0003:00000bc8       __scrt_native_startup_lock 0000000180012bc8     MSVCRT:utility.obj
 0003:00000c08       __scrt_debugger_hook_flag  0000000180012c08     MSVCRT:utility_desktop.obj
 0003:00000c0c       __favor                    0000000180012c0c     MSVCRT:cpu_disp.obj
 0003:00000c10       __dyn_tls_init_callback    0000000180012c10     <common>

 entry point at        0001:00009090

 Static symbols

 0000:fffea000       .debug$S                   0000000180000000     nio.exp
 0000:fffea000       .debug$S                   0000000180000000     vcruntime:VCRUNTIME140.dll
 0000:fffea000       .debug$S                   0000000180000000     vcruntime:VCRUNTIME140.dll
 0000:fffea000       .debug$S                   0000000180000000     vcruntime:VCRUNTIME140.dll
 0000:fffea000       .debug$S                   0000000180000000     vcruntime:VCRUNTIME140.dll
 0000:fffea000       .debug$S                   0000000180000000     vcruntime:VCRUNTIME140.dll
 0000:fffea000       .debug$S                   0000000180000000     vcruntime:VCRUNTIME140.dll
 0000:fffea000       .debug$S                   0000000180000000     ucrt:api-ms-win-crt-heap-l1-1-0.dll
 0000:fffea000       .debug$S                   0000000180000000     ucrt:api-ms-win-crt-heap-l1-1-0.dll
 0000:fffea000       .debug$S                   0000000180000000     ucrt:api-ms-win-crt-runtime-l1-1-0.dll
 0000:fffea000       .debug$S                   0000000180000000     ucrt:api-ms-win-crt-runtime-l1-1-0.dll
 0000:fffea000       .debug$S                   0000000180000000     ucrt:api-ms-win-crt-runtime-l1-1-0.dll
 0000:fffea000       .debug$S                   0000000180000000     ucrt:api-ms-win-crt-runtime-l1-1-0.dll
 0000:fffea000       .debug$S                   0000000180000000     ucrt:api-ms-win-crt-runtime-l1-1-0.dll
 0000:fffea000       .debug$S                   0000000180000000     ucrt:api-ms-win-crt-runtime-l1-1-0.dll
 0000:fffea000       .debug$S                   0000000180000000     ucrt:api-ms-win-crt-runtime-l1-1-0.dll
 0000:fffea000       .debug$S                   0000000180000000     ucrt:api-ms-win-crt-runtime-l1-1-0.dll
 0000:fffea000       .debug$S                   0000000180000000     ucrt:api-ms-win-crt-runtime-l1-1-0.dll
 0000:fffea000       .debug$S                   0000000180000000     ucrt:api-ms-win-crt-runtime-l1-1-0.dll
 0000:fffea000       .debug$S                   0000000180000000     ucrt:api-ms-win-crt-runtime-l1-1-0.dll
 0000:fffea000       .debug$S                   0000000180000000     ucrt:api-ms-win-crt-runtime-l1-1-0.dll
 0000:fffea000       .debug$S                   0000000180000000     ucrt:api-ms-win-crt-runtime-l1-1-0.dll
 0000:fffea000       .debug$S                   0000000180000000     ucrt:api-ms-win-crt-runtime-l1-1-0.dll
 0000:fffea000       .debug$S                   0000000180000000     ucrt:api-ms-win-crt-string-l1-1-0.dll
 0000:fffea000       .debug$S                   0000000180000000     ucrt:api-ms-win-crt-string-l1-1-0.dll
 0000:fffea000       .debug$S                   0000000180000000     ucrt:api-ms-win-crt-string-l1-1-0.dll
 0000:fffea000       .debug$S                   0000000180000000     advapi32:ADVAPI32.dll
 0000:fffea000       .debug$S                   0000000180000000     advapi32:ADVAPI32.dll
 0000:fffea000       .debug$S                   0000000180000000     advapi32:ADVAPI32.dll
 0000:fffea000       .debug$S                   0000000180000000     advapi32:ADVAPI32.dll
 0000:fffea000       .debug$S                   0000000180000000     advapi32:ADVAPI32.dll
 0000:fffea000       .debug$S                   0000000180000000     advapi32:ADVAPI32.dll
 0000:fffea000       .debug$S                   0000000180000000     advapi32:ADVAPI32.dll
 0000:fffea000       .debug$S                   0000000180000000     advapi32:ADVAPI32.dll
 0000:fffea000       .debug$S                   0000000180000000     advapi32:ADVAPI32.dll
 0000:fffea000       .debug$S                   0000000180000000     advapi32:ADVAPI32.dll
 0000:fffea000       .debug$S                   0000000180000000     advapi32:ADVAPI32.dll
 0000:fffea000       .debug$S                   0000000180000000     advapi32:ADVAPI32.dll
 0000:fffea000       .debug$S                   0000000180000000     advapi32:ADVAPI32.dll
 0000:fffea000       .debug$S                   0000000180000000     advapi32:ADVAPI32.dll
 0000:fffea000       .debug$S                   0000000180000000     advapi32:ADVAPI32.dll
 0000:fffea000       .debug$S                   0000000180000000     advapi32:ADVAPI32.dll
 0000:fffea000       .debug$S                   0000000180000000     advapi32:ADVAPI32.dll
 0000:fffea000       .debug$S                   0000000180000000     advapi32:ADVAPI32.dll
 0000:fffea000       .debug$S                   0000000180000000     advapi32:ADVAPI32.dll
 0000:fffea000       .debug$S                   0000000180000000     advapi32:ADVAPI32.dll
 0000:fffea000       .debug$S                   0000000180000000     advapi32:ADVAPI32.dll
 0000:fffea000       .debug$S                   0000000180000000     advapi32:ADVAPI32.dll
 0000:fffea000       .debug$S                   0000000180000000     advapi32:ADVAPI32.dll
 0000:fffea000       .debug$S                   0000000180000000     advapi32:ADVAPI32.dll
 0000:fffea000       .debug$S                   0000000180000000     advapi32:ADVAPI32.dll
 0000:fffea000       .debug$S                   0000000180000000     advapi32:ADVAPI32.dll
 0000:fffea000       .debug$S                   0000000180000000     advapi32:ADVAPI32.dll
 0000:fffea000       .debug$S                   0000000180000000     advapi32:ADVAPI32.dll
 0000:fffea000       .debug$S                   0000000180000000     advapi32:ADVAPI32.dll
 0000:fffea000       .debug$S                   0000000180000000     kernel32:KERNEL32.dll
 0000:fffea000       .debug$S                   0000000180000000     kernel32:KERNEL32.dll
 0000:fffea000       .debug$S                   0000000180000000     kernel32:KERNEL32.dll
 0000:fffea000       .debug$S                   0000000180000000     kernel32:KERNEL32.dll
 0000:fffea000       .debug$S                   0000000180000000     kernel32:KERNEL32.dll
 0000:fffea000       .debug$S                   0000000180000000     kernel32:KERNEL32.dll
 0000:fffea000       .debug$S                   0000000180000000     kernel32:KERNEL32.dll
 0000:fffea000       .debug$S                   0000000180000000     kernel32:KERNEL32.dll
 0000:fffea000       .debug$S                   0000000180000000     kernel32:KERNEL32.dll
 0000:fffea000       .debug$S                   0000000180000000     kernel32:KERNEL32.dll
 0000:fffea000       .debug$S                   0000000180000000     kernel32:KERNEL32.dll
 0000:fffea000       .debug$S                   0000000180000000     kernel32:KERNEL32.dll
 0000:fffea000       .debug$S                   0000000180000000     kernel32:KERNEL32.dll
 0000:fffea000       .debug$S                   0000000180000000     kernel32:KERNEL32.dll
 0000:fffea000       .debug$S                   0000000180000000     kernel32:KERNEL32.dll
 0000:fffea000       .debug$S                   0000000180000000     kernel32:KERNEL32.dll
 0000:fffea000       .debug$S                   0000000180000000     kernel32:KERNEL32.dll
 0000:fffea000       .debug$S                   0000000180000000     kernel32:KERNEL32.dll
 0000:fffea000       .debug$S                   0000000180000000     kernel32:KERNEL32.dll
 0000:fffea000       .debug$S                   0000000180000000     kernel32:KERNEL32.dll
 0000:fffea000       .debug$S                   0000000180000000     kernel32:KERNEL32.dll
 0000:fffea000       .debug$S                   0000000180000000     kernel32:KERNEL32.dll
 0000:fffea000       .debug$S                   0000000180000000     kernel32:KERNEL32.dll
 0000:fffea000       .debug$S                   0000000180000000     kernel32:KERNEL32.dll
 0000:fffea000       .debug$S                   0000000180000000     kernel32:KERNEL32.dll
 0000:fffea000       .debug$S                   0000000180000000     kernel32:KERNEL32.dll
 0000:fffea000       .debug$S                   0000000180000000     kernel32:KERNEL32.dll
 0000:fffea000       .debug$S                   0000000180000000     kernel32:KERNEL32.dll
 0000:fffea000       .debug$S                   0000000180000000     kernel32:KERNEL32.dll
 0000:fffea000       .debug$S                   0000000180000000     kernel32:KERNEL32.dll
 0000:fffea000       .debug$S                   0000000180000000     kernel32:KERNEL32.dll
 0000:fffea000       .debug$S                   0000000180000000     kernel32:KERNEL32.dll
 0000:fffea000       .debug$S                   0000000180000000     kernel32:KERNEL32.dll
 0000:fffea000       .debug$S                   0000000180000000     kernel32:KERNEL32.dll
 0000:fffea000       .debug$S                   0000000180000000     kernel32:KERNEL32.dll
 0000:fffea000       .debug$S                   0000000180000000     kernel32:KERNEL32.dll
 0000:fffea000       .debug$S                   0000000180000000     kernel32:KERNEL32.dll
 0000:fffea000       .debug$S                   0000000180000000     kernel32:KERNEL32.dll
 0000:fffea000       .debug$S                   0000000180000000     kernel32:KERNEL32.dll
 0000:fffea000       .debug$S                   0000000180000000     kernel32:KERNEL32.dll
 0000:fffea000       .debug$S                   0000000180000000     kernel32:KERNEL32.dll
 0000:fffea000       .debug$S                   0000000180000000     kernel32:KERNEL32.dll
 0000:fffea000       .debug$S                   0000000180000000     kernel32:KERNEL32.dll
 0000:fffea000       .debug$S                   0000000180000000     kernel32:KERNEL32.dll
 0000:fffea000       .debug$S                   0000000180000000     kernel32:KERNEL32.dll
 0000:fffea000       .debug$S                   0000000180000000     kernel32:KERNEL32.dll
 0000:fffea000       .debug$S                   0000000180000000     kernel32:KERNEL32.dll
 0000:fffea000       .debug$S                   0000000180000000     kernel32:KERNEL32.dll
 0000:fffea000       .debug$S                   0000000180000000     kernel32:KERNEL32.dll
 0000:fffea000       .debug$S                   0000000180000000     kernel32:KERNEL32.dll
 0000:fffea000       .debug$S                   0000000180000000     kernel32:KERNEL32.dll
 0000:fffea000       .debug$S                   0000000180000000     kernel32:KERNEL32.dll
 0000:fffea000       .debug$S                   0000000180000000     kernel32:KERNEL32.dll
 0000:fffea000       .debug$S                   0000000180000000     kernel32:KERNEL32.dll
 0000:fffea000       .debug$S                   0000000180000000     kernel32:KERNEL32.dll
 0000:fffea000       .debug$S                   0000000180000000     kernel32:KERNEL32.dll
 0000:fffea000       .debug$S                   0000000180000000     kernel32:KERNEL32.dll
 0000:fffea000       .debug$S                   0000000180000000     kernel32:KERNEL32.dll
 0000:fffea000       .debug$S                   0000000180000000     kernel32:KERNEL32.dll
 0000:fffea000       .debug$S                   0000000180000000     kernel32:KERNEL32.dll
 0000:fffea000       .debug$S                   0000000180000000     kernel32:KERNEL32.dll
 0000:fffea000       .debug$S                   0000000180000000     kernel32:KERNEL32.dll
 0000:fffea000       .debug$S                   0000000180000000     kernel32:KERNEL32.dll
 0000:fffea000       .debug$S                   0000000180000000     kernel32:KERNEL32.dll
 0000:fffea000       .debug$S                   0000000180000000     kernel32:KERNEL32.dll
 0000:fffea000       .debug$S                   0000000180000000     kernel32:KERNEL32.dll
 0000:fffea000       .debug$S                   0000000180000000     kernel32:KERNEL32.dll
 0000:fffea000       .debug$S                   0000000180000000     kernel32:KERNEL32.dll
 0000:fffea000       .debug$S                   0000000180000000     kernel32:KERNEL32.dll
 0000:fffea000       .debug$S                   0000000180000000     kernel32:KERNEL32.dll
 0000:fffea000       .debug$S                   0000000180000000     kernel32:KERNEL32.dll
 0000:fffea000       .debug$S                   0000000180000000     kernel32:KERNEL32.dll
 0000:fffea000       .debug$S                   0000000180000000     kernel32:KERNEL32.dll
 0000:fffea000       .debug$S                   0000000180000000     kernel32:KERNEL32.dll
 0000:fffea000       .debug$S                   0000000180000000     kernel32:KERNEL32.dll
 0000:fffea000       .debug$S                   0000000180000000     kernel32:KERNEL32.dll
 0000:fffea000       .debug$S                   0000000180000000     kernel32:KERNEL32.dll
 0000:fffea000       .debug$S                   0000000180000000     kernel32:KERNEL32.dll
 0000:fffea000       .debug$S                   0000000180000000     kernel32:KERNEL32.dll
 0000:fffea000       .debug$S                   0000000180000000     kernel32:KERNEL32.dll
 0000:fffea000       .debug$S                   0000000180000000     kernel32:KERNEL32.dll
 0000:fffea000       .debug$S                   0000000180000000     kernel32:KERNEL32.dll
 0000:fffea000       .debug$S                   0000000180000000     kernel32:KERNEL32.dll
 0000:fffea000       .debug$S                   0000000180000000     kernel32:KERNEL32.dll
 0000:fffea000       .debug$S                   0000000180000000     kernel32:KERNEL32.dll
 0000:fffea000       .debug$S                   0000000180000000     kernel32:KERNEL32.dll
 0000:fffea000       .debug$S                   0000000180000000     kernel32:KERNEL32.dll
 0000:fffea000       .debug$S                   0000000180000000     kernel32:KERNEL32.dll
 0000:fffea000       .debug$S                   0000000180000000     kernel32:KERNEL32.dll
 0000:fffea000       .debug$S                   0000000180000000     kernel32:KERNEL32.dll
 0000:fffea000       .debug$S                   0000000180000000     kernel32:KERNEL32.dll
 0000:fffea000       .debug$S                   0000000180000000     mswsock:MSWSOCK.dll
 0000:fffea000       .debug$S                   0000000180000000     ws2_32:WS2_32.dll
 0000:fffea000       .debug$S                   0000000180000000     ws2_32:WS2_32.dll
 0000:fffea000       .debug$S                   0000000180000000     ws2_32:WS2_32.dll
 0000:fffea000       .debug$S                   0000000180000000     ws2_32:WS2_32.dll
 0000:fffea000       .debug$S                   0000000180000000     ws2_32:WS2_32.dll
 0000:fffea000       .debug$S                   0000000180000000     ws2_32:WS2_32.dll
 0000:fffea000       .debug$S                   0000000180000000     ws2_32:WS2_32.dll
 0000:fffea000       .debug$S                   0000000180000000     ws2_32:WS2_32.dll
 0000:fffea000       .debug$S                   0000000180000000     ws2_32:WS2_32.dll
 0000:fffea000       .debug$S                   0000000180000000     ws2_32:WS2_32.dll
 0000:fffea000       .debug$S                   0000000180000000     ws2_32:WS2_32.dll
 0000:fffea000       .debug$S                   0000000180000000     ws2_32:WS2_32.dll
 0000:fffea000       .debug$S                   0000000180000000     ws2_32:WS2_32.dll
 0000:fffea000       .debug$S                   0000000180000000     ws2_32:WS2_32.dll
 0000:fffea000       .debug$S                   0000000180000000     ws2_32:WS2_32.dll
 0000:fffea000       .debug$S                   0000000180000000     ws2_32:WS2_32.dll
 0000:fffea000       .debug$S                   0000000180000000     ws2_32:WS2_32.dll
 0000:fffea000       .debug$S                   0000000180000000     ws2_32:WS2_32.dll
 0000:fffea000       .debug$S                   0000000180000000     ws2_32:WS2_32.dll
 0000:fffea000       .debug$S                   0000000180000000     ws2_32:WS2_32.dll
 0000:fffea000       .debug$S                   0000000180000000     ws2_32:WS2_32.dll
 0000:fffea000       .debug$S                   0000000180000000     ws2_32:WS2_32.dll
 0000:fffea000       .debug$S                   0000000180000000     ws2_32:WS2_32.dll
 0000:fffea000       .debug$S                   0000000180000000     ws2_32:WS2_32.dll
 0000:fffea000       .debug$S                   0000000180000000     ws2_32:WS2_32.dll
 0000:fffea000       .debug$S                   0000000180000000     ws2_32:WS2_32.dll
 0000:fffea000       .debug$S                   0000000180000000     ws2_32:WS2_32.dll
 0000:fffea000       .debug$S                   0000000180000000     ws2_32:WS2_32.dll
 0000:fffea000       .debug$S                   0000000180000000     ws2_32:WS2_32.dll
 0000:fffea000       .debug$S                   0000000180000000     java:java.dll
 0000:fffea000       .debug$S                   0000000180000000     java:java.dll
 0000:fffea000       .debug$S                   0000000180000000     java:java.dll
 0000:fffea000       .debug$S                   0000000180000000     java:java.dll
 0000:fffea000       .debug$S                   0000000180000000     java:java.dll
 0000:fffea000       .debug$S                   0000000180000000     java:java.dll
 0000:fffea000       .debug$S                   0000000180000000     java:java.dll
 0000:fffea000       .debug$S                   0000000180000000     net:net.dll
 0000:fffea000       .debug$S                   0000000180000000     net:net.dll
 0000:fffea000       .debug$S                   0000000180000000     net:net.dll
 0000:fffea000       .debug$S                   0000000180000000     net:net.dll
 0000:fffea000       .debug$S                   0000000180000000     net:net.dll
 0000:fffea000       .debug$S                   0000000180000000     net:net.dll
 0000:fffea000       .debug$S                   0000000180000000     net:net.dll
 0000:fffea000       .debug$S                   0000000180000000     net:net.dll
 0000:fffea000       .debug$S                   0000000180000000     net:net.dll
 0000:fffea000       .debug$S                   0000000180000000     net:net.dll
 0000:fffea000       .debug$S                   0000000180000000     net:net.dll
 0001:00003260       setGroupSourceReqOption    0000000180004260 f   Net.obj
 0001:000066b0       throwWindowsException      00000001800076b0 f   WindowsNativeDispatcher.obj
 0001:00006b24       afd_create_device_handle   0000000180007b24 f   wepoll.obj
 0001:00006c1c       epoll__create              0000000180007c1c f   wepoll.obj
 0001:00006fa0       err__map_win_error_to_errno 0000000180007fa0 f   wepoll.obj
 0001:000073d8       err_check_handle           00000001800083d8 f   wepoll.obj
 0001:00007424       err_set_win_error          0000000180008424 f   wepoll.obj
 0001:0000744c       init                       000000018000844c f   wepoll.obj
 0001:00007484       init__once_callback        0000000180008484 f   wepoll.obj
 0001:00007530       nt_global_init             0000000180008530 f   wepoll.obj
 0001:00007628       poll_group__new            0000000180008628 f   wepoll.obj
 0001:000076d4       port__ctl_add              00000001800086d4 f   wepoll.obj
 0001:000078cc       port__feed_events          00000001800088cc f   wepoll.obj
 0001:00007a2c       port_ctl                   0000000180008a2c f   wepoll.obj
 0001:00007b94       port_delete                0000000180008b94 f   wepoll.obj
 0001:00007c5c       port_new                   0000000180008c5c f   wepoll.obj
 0001:00007d44       port_wait                  0000000180008d44 f   wepoll.obj
 0001:00007f40       sock__delete               0000000180008f40 f   wepoll.obj
 0001:000080b4       sock_update                00000001800090b4 f   wepoll.obj
 0001:000082d8       tree_add                   00000001800092d8 f   wepoll.obj
 0001:00008490       tree_del                   0000000180009490 f   wepoll.obj
 0001:000087e8       ts_tree_find_and_ref       00000001800097e8 f   wepoll.obj
 0001:0000884c       ws_get_base_socket         000000018000984c f   wepoll.obj
 0001:00008a40       $$000000                   0000000180009a40     MSVCRT:amdsecgs.obj
 0001:00008c28       capture_current_context    0000000180009c28 f   MSVCRT:gs_report.obj
 0001:00008c98       capture_previous_context   0000000180009c98 f   MSVCRT:gs_report.obj
 0001:00008d10       $$000000                   0000000180009d10     MSVCRT:chkstk.obj
 0001:00008d70       ?dllmain_crt_dispatch@@YAHQEAUHINSTANCE__@@KQEAX@Z 0000000180009d70 f   MSVCRT:dll_dllmain.obj
 0001:00008dc0       ?dllmain_crt_process_attach@@YAHQEAUHINSTANCE__@@QEAX@Z 0000000180009dc0 f   MSVCRT:dll_dllmain.obj
 0001:00008ed8       ?dllmain_crt_process_detach@@YAH_N@Z 0000000180009ed8 f   MSVCRT:dll_dllmain.obj
 0001:00008f5c       ?dllmain_dispatch@@YAHQEAUHINSTANCE__@@KQEAX@Z 0000000180009f5c f   MSVCRT:dll_dllmain.obj
 0001:000098f0       $$000000                   000000018000a8f0     MSVCRT:guard_dispatch.obj
 0001:00009910       $$000000                   000000018000a910     MSVCRT:guard_xfg_dispatch.obj
 0001:00009926       ?fin$0@?0??dllmain_crt_process_attach@@YAHQEAUHINSTANCE__@@QEAX@Z@4HA 000000018000a926 f   MSVCRT:dll_dllmain.obj
 0001:0000993d       ?fin$0@?0??dllmain_crt_process_detach@@YAH_N@Z@4HA 000000018000a93d f   MSVCRT:dll_dllmain.obj
 0001:00009956       ?fin$1@?0??dllmain_crt_process_detach@@YAH_N@Z@4HA 000000018000a956 f   MSVCRT:dll_dllmain.obj
 0001:0000996a       ?filt$0@?0??dllmain_dispatch@@YAHQEAUHINSTANCE__@@KQEAX@Z@4HA 000000018000a96a f   MSVCRT:dll_dllmain.obj
 0001:000099a0       __scrt_is_nonwritable_in_current_image$filt$0 000000018000a9a0 f   MSVCRT:utility.obj
 0002:00001230       GS_ExceptionPointers       000000018000c230     MSVCRT:gs_report.obj
 0002:000017e0       $unwind$purgeOutstandingICMP 000000018000c7e0     DatagramChannelImpl.obj
 0002:00001800       $unwind$Java_sun_nio_ch_DatagramChannelImpl_disconnect0 000000018000c800     DatagramChannelImpl.obj
 0002:00001800       $unwind$Java_sun_nio_ch_FileKey_init 000000018000c800     FileKey.obj
 0002:00001814       $unwind$Java_sun_nio_ch_DatagramChannelImpl_receive0 000000018000c814     DatagramChannelImpl.obj
 0002:0000182c       $unwind$Java_sun_nio_ch_DatagramChannelImpl_send0 000000018000c82c     DatagramChannelImpl.obj
 0002:0000182c       $unwind$Java_sun_nio_ch_SocketDispatcher_close0 000000018000c82c     SocketDispatcher.obj
 0002:0000182c       $unwind$Java_sun_nio_ch_UnixDomainSockets_socket0 000000018000c82c     UnixDomainSockets.obj
 0002:0000182c       $unwind$Java_sun_nio_ch_WindowsAsynchronousFileChannelImpl_lockFile 000000018000c82c     WindowsAsynchronousFileChannelImpl.obj
 0002:00001838       $unwind$Java_sun_nio_ch_DatagramDispatcher_read0 000000018000c838     DatagramDispatcher.obj
 0002:0000184c       $unwind$Java_sun_nio_ch_DatagramDispatcher_readv0 000000018000c84c     DatagramDispatcher.obj
 0002:0000184c       $unwind$Java_sun_nio_ch_SocketDispatcher_readv0 000000018000c84c     SocketDispatcher.obj
 0002:00001864       $unwind$Java_sun_nio_ch_DatagramDispatcher_write0 000000018000c864     DatagramDispatcher.obj
 0002:00001878       $unwind$Java_sun_nio_ch_DatagramDispatcher_writev0 000000018000c878     DatagramDispatcher.obj
 0002:00001890       $unwind$Java_sun_nio_ch_FileDispatcherImpl_duplicateHandle 000000018000c890     FileDispatcherImpl.obj
 0002:00001890       $unwind$Java_sun_nio_ch_FileDispatcherImpl_read0 000000018000c890     FileDispatcherImpl.obj
 0002:00001890       $unwind$Java_sun_nio_ch_Net_setInterface4 000000018000c890     Net.obj
 0002:0000189c       $unwind$Java_sun_nio_ch_FileDispatcherImpl_pread0 000000018000c89c     FileDispatcherImpl.obj
 0002:0000189c       $unwind$Java_sun_nio_ch_FileDispatcherImpl_pwrite0 000000018000c89c     FileDispatcherImpl.obj
 0002:0000189c       $unwind$Java_sun_nio_ch_FileDispatcherImpl_write0 000000018000c89c     FileDispatcherImpl.obj
 0002:000018ac       $unwind$Java_sun_nio_ch_FileDispatcherImpl_readv0 000000018000c8ac     FileDispatcherImpl.obj
 0002:000018c4       $unwind$Java_sun_nio_ch_FileDispatcherImpl_writev0 000000018000c8c4     FileDispatcherImpl.obj
 0002:000018e0       $unwind$Java_sun_nio_ch_FileDispatcherImpl_seek0 000000018000c8e0     FileDispatcherImpl.obj
 0002:000018e0       $unwind$Java_sun_nio_ch_FileDispatcherImpl_truncate0 000000018000c8e0     FileDispatcherImpl.obj
 0002:000018e0       $unwind$Java_sun_nio_ch_IOUtil_configureBlocking 000000018000c8e0     IOUtil.obj
 0002:000018e0       $unwind$Java_sun_nio_ch_IOUtil_initIDs 000000018000c8e0     IOUtil.obj
 0002:000018e0       $unwind$Java_sun_nio_ch_Iocp_createIoCompletionPort 000000018000c8e0     Iocp.obj
 0002:000018e0       $unwind$Java_sun_nio_ch_Iocp_initIDs 000000018000c8e0     Iocp.obj
 0002:000018e0       $unwind$Java_sun_nio_ch_Net_initIDs 000000018000c8e0     Net.obj
 0002:000018e0       $unwind$Java_sun_nio_ch_Net_listen 000000018000c8e0     Net.obj
 0002:000018e0       $unwind$Java_sun_nio_ch_Net_shutdown 000000018000c8e0     Net.obj
 0002:000018e0       $unwind$Java_sun_nio_ch_WEPoll_create 000000018000c8e0     WEPollNatives.obj
 0002:000018e0       $unwind$Java_sun_nio_fs_WindowsNativeDispatcher_ConvertSidToStringSid 000000018000c8e0     WindowsNativeDispatcher.obj
 0002:000018e0       $unwind$Java_sun_nio_fs_WindowsNativeDispatcher_CreateEvent 000000018000c8e0     WindowsNativeDispatcher.obj
 0002:000018e0       $unwind$Java_sun_nio_fs_WindowsNativeDispatcher_CreateIoCompletionPort 000000018000c8e0     WindowsNativeDispatcher.obj
 0002:000018e0       $unwind$Java_sun_nio_fs_WindowsNativeDispatcher_FindFirstFile1 000000018000c8e0     WindowsNativeDispatcher.obj
 0002:000018e0       $unwind$Java_sun_nio_fs_WindowsNativeDispatcher_GetFileAttributes0 000000018000c8e0     WindowsNativeDispatcher.obj
 0002:000018e0       $unwind$Java_sun_nio_fs_WindowsNativeDispatcher_GetLogicalDrives 000000018000c8e0     WindowsNativeDispatcher.obj
 0002:000018e0       $unwind$_RTC_Initialize    000000018000c8e0     MSVCRT:initsect.obj
 0002:000018e0       $unwind$_RTC_Terminate     000000018000c8e0     MSVCRT:initsect.obj
 0002:000018ec       $unwind$Java_sun_nio_ch_FileDispatcherImpl_close0 000000018000c8ec     FileDispatcherImpl.obj
 0002:000018ec       $unwind$Java_sun_nio_ch_FileDispatcherImpl_force0 000000018000c8ec     FileDispatcherImpl.obj
 0002:000018ec       $unwind$Java_sun_nio_ch_FileDispatcherImpl_size0 000000018000c8ec     FileDispatcherImpl.obj
 0002:000018ec       $unwind$Java_sun_nio_ch_FileDispatcherImpl_unmap0 000000018000c8ec     FileDispatcherImpl.obj
 0002:000018ec       $unwind$Java_sun_nio_ch_Iocp_postQueuedCompletionStatus 000000018000c8ec     Iocp.obj
 0002:000018ec       $unwind$Java_sun_nio_ch_Net_available 000000018000c8ec     Net.obj
 0002:000018ec       $unwind$Java_sun_nio_ch_WEPoll_wait 000000018000c8ec     WEPollNatives.obj
 0002:000018ec       $unwind$Java_sun_nio_ch_WindowsAsynchronousServerSocketChannelImpl_closesocket0 000000018000c8ec     WindowsAsynchronousServerSocketChannelImpl.obj
 0002:000018ec       $unwind$Java_sun_nio_ch_WindowsAsynchronousSocketChannelImpl_closesocket0 000000018000c8ec     WindowsAsynchronousSocketChannelImpl.obj
 0002:000018ec       $unwind$Java_sun_nio_ch_WindowsAsynchronousSocketChannelImpl_shutdown0 000000018000c8ec     WindowsAsynchronousSocketChannelImpl.obj
 0002:000018ec       $unwind$Java_sun_nio_fs_WindowsNativeDispatcher_CancelIo 000000018000c8ec     WindowsNativeDispatcher.obj
 0002:000018ec       $unwind$Java_sun_nio_fs_WindowsNativeDispatcher_ConvertStringSidToSid0 000000018000c8ec     WindowsNativeDispatcher.obj
 0002:000018ec       $unwind$Java_sun_nio_fs_WindowsNativeDispatcher_CreateHardLink0 000000018000c8ec     WindowsNativeDispatcher.obj
 0002:000018ec       $unwind$Java_sun_nio_fs_WindowsNativeDispatcher_CreateSymbolicLink0 000000018000c8ec     WindowsNativeDispatcher.obj
 0002:000018ec       $unwind$Java_sun_nio_fs_WindowsNativeDispatcher_DeleteFile0 000000018000c8ec     WindowsNativeDispatcher.obj
 0002:000018ec       $unwind$Java_sun_nio_fs_WindowsNativeDispatcher_FindClose 000000018000c8ec     WindowsNativeDispatcher.obj
 0002:000018ec       $unwind$Java_sun_nio_fs_WindowsNativeDispatcher_GetAce 000000018000c8ec     WindowsNativeDispatcher.obj
 0002:000018ec       $unwind$Java_sun_nio_fs_WindowsNativeDispatcher_GetFileAttributesEx0 000000018000c8ec     WindowsNativeDispatcher.obj
 0002:000018ec       $unwind$Java_sun_nio_fs_WindowsNativeDispatcher_GetFileInformationByHandle0 000000018000c8ec     WindowsNativeDispatcher.obj
 0002:000018ec       $unwind$Java_sun_nio_fs_WindowsNativeDispatcher_GetFileInformationByName0 000000018000c8ec     WindowsNativeDispatcher.obj
 0002:000018ec       $unwind$Java_sun_nio_fs_WindowsNativeDispatcher_GetFileSizeEx 000000018000c8ec     WindowsNativeDispatcher.obj
 0002:000018ec       $unwind$Java_sun_nio_fs_WindowsNativeDispatcher_GetSecurityDescriptorOwner 000000018000c8ec     WindowsNativeDispatcher.obj
 0002:000018ec       $unwind$Java_sun_nio_fs_WindowsNativeDispatcher_InitializeAcl 000000018000c8ec     WindowsNativeDispatcher.obj
 0002:000018ec       $unwind$Java_sun_nio_fs_WindowsNativeDispatcher_InitializeSecurityDescriptor 000000018000c8ec     WindowsNativeDispatcher.obj
 0002:000018ec       $unwind$Java_sun_nio_fs_WindowsNativeDispatcher_MoveFileEx0 000000018000c8ec     WindowsNativeDispatcher.obj
 0002:000018ec       $unwind$Java_sun_nio_fs_WindowsNativeDispatcher_OpenProcessToken 000000018000c8ec     WindowsNativeDispatcher.obj
 0002:000018ec       $unwind$Java_sun_nio_fs_WindowsNativeDispatcher_OpenThreadToken 000000018000c8ec     WindowsNativeDispatcher.obj
 0002:000018ec       $unwind$Java_sun_nio_fs_WindowsNativeDispatcher_PostQueuedCompletionStatus 000000018000c8ec     WindowsNativeDispatcher.obj
 0002:000018ec       $unwind$Java_sun_nio_fs_WindowsNativeDispatcher_RemoveDirectory0 000000018000c8ec     WindowsNativeDispatcher.obj
 0002:000018ec       $unwind$Java_sun_nio_fs_WindowsNativeDispatcher_SetEndOfFile 000000018000c8ec     WindowsNativeDispatcher.obj
 0002:000018ec       $unwind$Java_sun_nio_fs_WindowsNativeDispatcher_SetFileAttributes0 000000018000c8ec     WindowsNativeDispatcher.obj
 0002:000018ec       $unwind$Java_sun_nio_fs_WindowsNativeDispatcher_SetFileSecurity0 000000018000c8ec     WindowsNativeDispatcher.obj
 0002:000018ec       $unwind$Java_sun_nio_fs_WindowsNativeDispatcher_SetSecurityDescriptorDacl 000000018000c8ec     WindowsNativeDispatcher.obj
 0002:000018ec       $unwind$Java_sun_nio_fs_WindowsNativeDispatcher_SetSecurityDescriptorOwner 000000018000c8ec     WindowsNativeDispatcher.obj
 0002:000018ec       $unwind$Java_sun_nio_fs_WindowsNativeDispatcher_SetThreadToken 000000018000c8ec     WindowsNativeDispatcher.obj
 0002:000018ec       $unwind$throwWindowsException 000000018000c8ec     WindowsNativeDispatcher.obj
 0002:000018ec       $unwind$err_check_handle   000000018000c8ec     wepoll.obj
 0002:000018ec       $unwind$err_set_win_error  000000018000c8ec     wepoll.obj
 0002:000018ec       $unwind$nt_global_init     000000018000c8ec     wepoll.obj
 0002:000018ec       $unwind$__raise_securityfailure 000000018000c8ec     MSVCRT:gs_report.obj
 0002:000018ec       $unwind$__scrt_initialize_crt 000000018000c8ec     MSVCRT:utility.obj
 0002:000018ec       $unwind$__scrt_initialize_onexit_tables 000000018000c8ec     MSVCRT:utility.obj
 0002:000018ec       $unwind$__scrt_release_startup_lock 000000018000c8ec     MSVCRT:utility.obj
 0002:000018ec       $unwind$__scrt_uninitialize_crt 000000018000c8ec     MSVCRT:utility.obj
 0002:000018f4       $unwind$Java_sun_nio_ch_FileDispatcherImpl_available0 000000018000c8f4     FileDispatcherImpl.obj
 0002:000018f4       $unwind$sockaddrToUnixAddressBytes 000000018000c8f4     UnixDomainSockets.obj
 0002:00001908       $unwind$Java_sun_nio_ch_FileDispatcherImpl_isOther0 000000018000c908     FileDispatcherImpl.obj
 0002:00001924       $unwind$Java_sun_nio_ch_FileDispatcherImpl_lock0 000000018000c924     FileDispatcherImpl.obj
 0002:00001924       $unwind$Java_sun_nio_ch_FileDispatcherImpl_release0 000000018000c924     FileDispatcherImpl.obj
 0002:00001934       $unwind$Java_sun_nio_ch_FileDispatcherImpl_allocationGranularity0 000000018000c934     FileDispatcherImpl.obj
 0002:0000193c       $unwind$Java_sun_nio_ch_FileDispatcherImpl_map0 000000018000c93c     FileDispatcherImpl.obj
 0002:00001958       $unwind$Java_sun_nio_ch_FileDispatcherImpl_transferTo0 000000018000c958     FileDispatcherImpl.obj
 0002:0000196c       $unwind$Java_sun_nio_ch_FileDispatcherImpl_setDirect0 000000018000c96c     FileDispatcherImpl.obj
 0002:0000197c       $unwind$convertLongReturnVal 000000018000c97c     IOUtil.obj
 0002:0000197c       $unwind$convertReturnVal   000000018000c97c     IOUtil.obj
 0002:0000197c       $unwind$Java_sun_nio_ch_Net_isIPv6Available0 000000018000c97c     Net.obj
 0002:0000197c       $unwind$Java_sun_nio_ch_WindowsSelectorImpl_setWakeupSocket0 000000018000c97c     WindowsSelectorImpl.obj
 0002:0000197c       $unwind$epoll_create1      000000018000c97c     wepoll.obj
 0002:0000197c       $unwind$init               000000018000c97c     wepoll.obj
 0002:0000197c       $unwind$__scrt_initialize_default_local_stdio_options 000000018000c97c     MSVCRT:default_local_stdio_options.obj
 0002:0000197c       $unwind$?dllmain_crt_dispatch@@YAHQEAUHINSTANCE__@@KQEAX@Z 000000018000c97c     MSVCRT:dll_dllmain.obj
 0002:0000197c       $unwind$DllMain            000000018000c97c     MSVCRT:dll_dllmain_stub.obj
 0002:0000197c       $unwind$__report_rangecheckfailure 000000018000c97c     MSVCRT:gs_report.obj
 0002:0000197c       $unwind$__GSHandlerCheck   000000018000c97c     MSVCRT:gshandler.obj
 0002:0000197c       $unwind$__scrt_acquire_startup_lock 000000018000c97c     MSVCRT:utility.obj
 0002:0000197c       $unwind$__scrt_dllmain_after_initialize_c 000000018000c97c     MSVCRT:utility.obj
 0002:0000197c       $unwind$__scrt_dllmain_before_initialize_c 000000018000c97c     MSVCRT:utility.obj
 0002:0000197c       $unwind$__scrt_dllmain_crt_thread_attach 000000018000c97c     MSVCRT:utility.obj
 0002:0000197c       $unwind$__scrt_dllmain_crt_thread_detach 000000018000c97c     MSVCRT:utility.obj
 0002:0000197c       $unwind$__scrt_dllmain_uninitialize_c 000000018000c97c     MSVCRT:utility.obj
 0002:0000197c       $unwind$__scrt_dllmain_uninitialize_critical 000000018000c97c     MSVCRT:utility.obj
 0002:00001984       $unwind$Java_sun_nio_ch_IOUtil_write1 000000018000c984     IOUtil.obj
 0002:00001990       $unwind$Java_sun_nio_ch_IOUtil_drain 000000018000c990     IOUtil.obj
 0002:000019a8       $unwind$Java_sun_nio_ch_Iocp_getQueuedCompletionStatus 000000018000c9a8     Iocp.obj
 0002:000019a8       $unwind$Java_sun_nio_fs_WindowsNativeDispatcher_GetQueuedCompletionStatus0 000000018000c9a8     WindowsNativeDispatcher.obj
 0002:000019b4       $unwind$Java_sun_nio_ch_Iocp_getErrorMessage 000000018000c9b4     Iocp.obj
 0002:000019b4       $unwind$Java_sun_nio_fs_WindowsNativeDispatcher_FormatMessage 000000018000c9b4     WindowsNativeDispatcher.obj
 0002:000019cc       $unwind$MappedMemoryUtils_force0 000000018000c9cc     MappedMemoryUtils.obj
 0002:000019cc       $unwind$epoll_ctl          000000018000c9cc     wepoll.obj
 0002:000019cc       $unwind$epoll_wait         000000018000c9cc     wepoll.obj
 0002:000019cc       $unwind$poll_group__new    000000018000c9cc     wepoll.obj
 0002:000019cc       $unwind$port__feed_events  000000018000c9cc     wepoll.obj
 0002:000019cc       $unwind$port_ctl           000000018000c9cc     wepoll.obj
 0002:000019e4       $unwind$Java_sun_nio_ch_Net_socket0 000000018000c9e4     Net.obj
 0002:000019f4       $unwind$Java_sun_nio_ch_Net_bind0 000000018000c9f4     Net.obj
 0002:00001a08       $unwind$Java_sun_nio_ch_Net_connect0 000000018000ca08     Net.obj
 0002:00001a2c       $unwind$Java_sun_nio_ch_Net_accept 000000018000ca2c     Net.obj
 0002:00001a44       $unwind$Java_sun_nio_ch_Net_localInetAddress 000000018000ca44     Net.obj
 0002:00001a44       $unwind$Java_sun_nio_ch_Net_localPort 000000018000ca44     Net.obj
 0002:00001a44       $unwind$Java_sun_nio_ch_Net_remoteInetAddress 000000018000ca44     Net.obj
 0002:00001a44       $unwind$Java_sun_nio_ch_Net_remotePort 000000018000ca44     Net.obj
 0002:00001a54       $unwind$Java_sun_nio_ch_Net_getIntOption0 000000018000ca54     Net.obj
 0002:00001a64       $unwind$Java_sun_nio_ch_Net_setIntOption0 000000018000ca64     Net.obj
 0002:00001a70       $unwind$Java_sun_nio_ch_Net_poll 000000018000ca70     Net.obj
 0002:00001a94       $unwind$Java_sun_nio_ch_Net_pollConnect 000000018000ca94     Net.obj
 0002:00001ab0       $unwind$Java_sun_nio_ch_Net_sendOOB 000000018000cab0     Net.obj
 0002:00001ab8       $unwind$Java_sun_nio_ch_Net_discardOOB 000000018000cab8     Net.obj
 0002:00001ad0       $unwind$Java_sun_nio_ch_Net_joinOrDrop4 000000018000cad0     Net.obj
 0002:00001aec       $unwind$Java_sun_nio_ch_Net_blockOrUnblock4 000000018000caec     Net.obj
 0002:00001b04       $unwind$Java_sun_nio_ch_Net_joinOrDrop6 000000018000cb04     Net.obj
 0002:00001b18       $unwind$Java_sun_nio_ch_Net_blockOrUnblock6 000000018000cb18     Net.obj
 0002:00001b18       $unwind$Java_sun_nio_ch_WindowsAsynchronousFileChannelImpl_readFile 000000018000cb18     WindowsAsynchronousFileChannelImpl.obj
 0002:00001b18       $unwind$Java_sun_nio_ch_WindowsAsynchronousFileChannelImpl_writeFile 000000018000cb18     WindowsAsynchronousFileChannelImpl.obj
 0002:00001b18       $unwind$Java_sun_nio_ch_WindowsAsynchronousServerSocketChannelImpl_updateAcceptContext 000000018000cb18     WindowsAsynchronousServerSocketChannelImpl.obj
 0002:00001b18       $unwind$Java_sun_nio_ch_WindowsAsynchronousSocketChannelImpl_updateConnectContext 000000018000cb18     WindowsAsynchronousSocketChannelImpl.obj
 0002:00001b18       $unwind$Java_sun_nio_fs_WindowsNativeDispatcher_AddAccessAllowedAceEx 000000018000cb18     WindowsNativeDispatcher.obj
 0002:00001b18       $unwind$Java_sun_nio_fs_WindowsNativeDispatcher_AddAccessDeniedAceEx 000000018000cb18     WindowsNativeDispatcher.obj
 0002:00001b18       $unwind$Java_sun_nio_fs_WindowsNativeDispatcher_CopyFileEx0 000000018000cb18     WindowsNativeDispatcher.obj
 0002:00001b18       $unwind$Java_sun_nio_fs_WindowsNativeDispatcher_DuplicateTokenEx 000000018000cb18     WindowsNativeDispatcher.obj
 0002:00001b18       $unwind$Java_sun_nio_fs_WindowsNativeDispatcher_GetFileSecurity0 000000018000cb18     WindowsNativeDispatcher.obj
 0002:00001b18       $unwind$Java_sun_nio_fs_WindowsNativeDispatcher_GetOverlappedResult 000000018000cb18     WindowsNativeDispatcher.obj
 0002:00001b18       $unwind$Java_sun_nio_fs_WindowsNativeDispatcher_GetSecurityDescriptorDacl 000000018000cb18     WindowsNativeDispatcher.obj
 0002:00001b18       $unwind$Java_sun_nio_fs_WindowsNativeDispatcher_GetTokenInformation 000000018000cb18     WindowsNativeDispatcher.obj
 0002:00001b20       $unwind$Java_sun_nio_ch_Net_getInterface4 000000018000cb20     Net.obj
 0002:00001b20       $unwind$Java_sun_nio_ch_Net_getInterface6 000000018000cb20     Net.obj
 0002:00001b20       $unwind$Java_sun_nio_fs_WindowsNativeDispatcher_CreateDirectory0 000000018000cb20     WindowsNativeDispatcher.obj
 0002:00001b20       $unwind$Java_sun_nio_fs_WindowsNativeDispatcher_ReadDirectoryChangesW 000000018000cb20     WindowsNativeDispatcher.obj
 0002:00001b28       $unwind$Java_sun_nio_ch_Net_setInterface6 000000018000cb28     Net.obj
 0002:00001b30       $unwind$setGroupSourceReqOption 000000018000cb30     Net.obj
 0002:00001b4c       $unwind$Java_sun_nio_fs_RegistryFileTypeDetector_queryStringValue 000000018000cb4c     RegistryFileTypeDetector.obj
 0002:00001b64       $unwind$Java_sun_nio_ch_SocketDispatcher_read0 000000018000cb64     SocketDispatcher.obj
 0002:00001b70       $unwind$Java_sun_nio_ch_SocketDispatcher_write0 000000018000cb70     SocketDispatcher.obj
 0002:00001b84       $unwind$Java_sun_nio_ch_SocketDispatcher_writev0 000000018000cb84     SocketDispatcher.obj
 0002:00001b9c       $unwind$unixSocketAddressToSockaddr 000000018000cb9c     UnixDomainSockets.obj
 0002:00001bb4       $unwind$Java_sun_nio_ch_UnixDomainSockets_init 000000018000cbb4     UnixDomainSockets.obj
 0002:00001bcc       $unwind$Java_sun_nio_ch_UnixDomainSockets_bind0 000000018000cbcc     UnixDomainSockets.obj
 0002:00001be4       $unwind$Java_sun_nio_ch_UnixDomainSockets_connect0 000000018000cbe4     UnixDomainSockets.obj
 0002:00001bfc       $unwind$Java_sun_nio_ch_UnixDomainSockets_accept0 000000018000cbfc     UnixDomainSockets.obj
 0002:00001c18       $unwind$Java_sun_nio_ch_UnixDomainSockets_localAddress0 000000018000cc18     UnixDomainSockets.obj
 0002:00001c2c       $unwind$Java_sun_nio_ch_WEPoll_ctl 000000018000cc2c     WEPollNatives.obj
 0002:00001c34       $unwind$Java_sun_nio_ch_WindowsAsynchronousServerSocketChannelImpl_initIDs 000000018000cc34     WindowsAsynchronousServerSocketChannelImpl.obj
 0002:00001c34       $unwind$Java_sun_nio_ch_WindowsAsynchronousSocketChannelImpl_initIDs 000000018000cc34     WindowsAsynchronousSocketChannelImpl.obj
 0002:00001c4c       $unwind$Java_sun_nio_ch_WindowsAsynchronousServerSocketChannelImpl_accept0 000000018000cc4c     WindowsAsynchronousServerSocketChannelImpl.obj
 0002:00001c4c       $unwind$Java_sun_nio_ch_WindowsAsynchronousSocketChannelImpl_read0 000000018000cc4c     WindowsAsynchronousSocketChannelImpl.obj
 0002:00001c60       $unwind$Java_sun_nio_ch_WindowsAsynchronousSocketChannelImpl_connect0 000000018000cc60     WindowsAsynchronousSocketChannelImpl.obj
 0002:00001c74       $unwind$Java_sun_nio_ch_WindowsAsynchronousSocketChannelImpl_write0 000000018000cc74     WindowsAsynchronousSocketChannelImpl.obj
 0002:00001c88       $unwind$Java_sun_nio_fs_WindowsNativeDispatcher_CreateFile0 000000018000cc88     WindowsNativeDispatcher.obj
 0002:00001c88       $unwind$ws_get_base_socket 000000018000cc88     wepoll.obj
 0002:00001c94       $unwind$Java_sun_nio_fs_WindowsNativeDispatcher_DeviceIoControlGetReparsePoint 000000018000cc94     WindowsNativeDispatcher.obj
 0002:00001c94       $unwind$Java_sun_nio_fs_WindowsNativeDispatcher_DeviceIoControlSetSparse 000000018000cc94     WindowsNativeDispatcher.obj
 0002:00001c9c       $unwind$Java_sun_nio_fs_WindowsNativeDispatcher_FindFirstFile0 000000018000cc9c     WindowsNativeDispatcher.obj
 0002:00001cb8       $unwind$Java_sun_nio_fs_WindowsNativeDispatcher_FindNextFile0 000000018000ccb8     WindowsNativeDispatcher.obj
 0002:00001cb8       $unwind$Java_sun_nio_fs_WindowsNativeDispatcher_LookupPrivilegeValue0 000000018000ccb8     WindowsNativeDispatcher.obj
 0002:00001cb8       $unwind$port_new           000000018000ccb8     wepoll.obj
 0002:00001cb8       $unwind$ts_tree_find_and_ref 000000018000ccb8     wepoll.obj
 0002:00001cb8       $unwind$_DllMainCRTStartup 000000018000ccb8     MSVCRT:dll_dllmain.obj
 0002:00001cc8       $unwind$Java_sun_nio_fs_WindowsNativeDispatcher_FindFirstStream0 000000018000ccc8     WindowsNativeDispatcher.obj
 0002:00001ce4       $unwind$Java_sun_nio_fs_WindowsNativeDispatcher_FindNextStream0 000000018000cce4     WindowsNativeDispatcher.obj
 0002:00001cfc       $unwind$Java_sun_nio_fs_WindowsNativeDispatcher_SetFileTime0 000000018000ccfc     WindowsNativeDispatcher.obj
 0002:00001d08       $unwind$Java_sun_nio_fs_WindowsNativeDispatcher_GetVolumeInformation0 000000018000cd08     WindowsNativeDispatcher.obj
 0002:00001d20       $unwind$Java_sun_nio_fs_WindowsNativeDispatcher_GetDiskFreeSpaceEx0 000000018000cd20     WindowsNativeDispatcher.obj
 0002:00001d2c       $unwind$Java_sun_nio_fs_WindowsNativeDispatcher_GetDiskFreeSpace0 000000018000cd2c     WindowsNativeDispatcher.obj
 0002:00001d38       $unwind$Java_sun_nio_fs_WindowsNativeDispatcher_GetVolumePathName0 000000018000cd38     WindowsNativeDispatcher.obj
 0002:00001d50       $unwind$Java_sun_nio_fs_WindowsNativeDispatcher_GetAclInformation0 000000018000cd50     WindowsNativeDispatcher.obj
 0002:00001d64       $unwind$Java_sun_nio_fs_WindowsNativeDispatcher_LookupAccountSid0 000000018000cd64     WindowsNativeDispatcher.obj
 0002:00001d80       $unwind$Java_sun_nio_fs_WindowsNativeDispatcher_LookupAccountName0 000000018000cd80     WindowsNativeDispatcher.obj
 0002:00001d94       $unwind$Java_sun_nio_fs_WindowsNativeDispatcher_AdjustTokenPrivileges 000000018000cd94     WindowsNativeDispatcher.obj
 0002:00001da4       $unwind$Java_sun_nio_fs_WindowsNativeDispatcher_AccessCheck 000000018000cda4     WindowsNativeDispatcher.obj
 0002:00001dbc       $unwind$Java_sun_nio_fs_WindowsNativeDispatcher_GetFinalPathNameByHandle 000000018000cdbc     WindowsNativeDispatcher.obj
 0002:00001dbc       $unwind$Java_sun_nio_fs_WindowsNativeDispatcher_GetFullPathName0 000000018000cdbc     WindowsNativeDispatcher.obj
 0002:00001ddc       $unwind$Java_sun_nio_fs_WindowsNativeDispatcher_init 000000018000cddc     WindowsNativeDispatcher.obj
 0002:00001df4       $unwind$Java_sun_nio_ch_WindowsSelectorImpl_resetWakeupSocket0 000000018000cdf4     WindowsSelectorImpl.obj
 0002:00001e0c       $unwind$Java_sun_nio_ch_WindowsSelectorImpl_00024SubSelector_poll0 000000018000ce0c     WindowsSelectorImpl.obj
 0002:00001e34       $unwind$JNI_OnLoad         000000018000ce34     nio_util.obj
 0002:00001e34       $unwind$epoll__create      000000018000ce34     wepoll.obj
 0002:00001e40       $unwind$epoll_close        000000018000ce40     wepoll.obj
 0002:00001e40       $unwind$port_delete        000000018000ce40     wepoll.obj
 0002:00001e40       $unwind$__scrt_dllmain_exception_filter 000000018000ce40     MSVCRT:utility.obj
 0002:00001e54       $unwind$afd_create_device_handle 000000018000ce54     wepoll.obj
 0002:00001e68       $unwind$port_wait          000000018000ce68     wepoll.obj
 0002:00001e88       $unwind$tree_del           000000018000ce88     wepoll.obj
 0002:00001e94       $unwind$init__once_callback 000000018000ce94     wepoll.obj
 0002:00001ea4       $unwind$sock_update        000000018000cea4     wepoll.obj
 0002:00001eb8       $unwind$port__ctl_add      000000018000ceb8     wepoll.obj
 0002:00001ed4       $unwind$sock__delete       000000018000ced4     wepoll.obj
 0002:00001ef0       $unwind$__GSHandlerCheckCommon 000000018000cef0     MSVCRT:gshandler.obj
 0002:00001ef8       $xdatasym                  000000018000cef8     MSVCRT:amdsecgs.obj
 0002:00001efc       $unwind$__report_securityfailure 000000018000cefc     MSVCRT:gs_report.obj
 0002:00001f04       $unwind$__report_gsfailure 000000018000cf04     MSVCRT:gs_report.obj
 0002:00001f0c       $unwind$capture_current_context 000000018000cf0c     MSVCRT:gs_report.obj
 0002:00001f18       $unwind$capture_previous_context 000000018000cf18     MSVCRT:gs_report.obj
 0002:00001f28       $xdatasym                  000000018000cf28     MSVCRT:chkstk.obj
 0002:00001f30       $unwind$?dllmain_crt_process_attach@@YAHQEAUHINSTANCE__@@QEAX@Z 000000018000cf30     MSVCRT:dll_dllmain.obj
 0002:00001f6c       $unwind$?fin$0@?0??dllmain_crt_process_attach@@YAHQEAUHINSTANCE__@@QEAX@Z@4HA 000000018000cf6c     MSVCRT:dll_dllmain.obj
 0002:00001f6c       $unwind$?fin$0@?0??dllmain_crt_process_detach@@YAH_N@Z@4HA 000000018000cf6c     MSVCRT:dll_dllmain.obj
 0002:00001f6c       $unwind$?fin$1@?0??dllmain_crt_process_detach@@YAH_N@Z@4HA 000000018000cf6c     MSVCRT:dll_dllmain.obj
 0002:00001f74       $unwind$?dllmain_crt_process_detach@@YAH_N@Z 000000018000cf74     MSVCRT:dll_dllmain.obj
 0002:00001fc8       $unwind$?dllmain_dispatch@@YAHQEAUHINSTANCE__@@KQEAX@Z 000000018000cfc8     MSVCRT:dll_dllmain.obj
 0002:00001ff0       $unwind$?filt$0@?0??dllmain_dispatch@@YAHQEAUHINSTANCE__@@KQEAX@Z@4HA 000000018000cff0     MSVCRT:dll_dllmain.obj
 0002:00001ff8       $unwind$__security_init_cookie 000000018000cff8     MSVCRT:gs_support.obj
 0002:00002004       $unwind$__scrt_is_nonwritable_in_current_image 000000018000d004     MSVCRT:utility.obj
 0002:00002024       $unwind$__scrt_is_nonwritable_in_current_image$filt$0 000000018000d024     MSVCRT:utility.obj
 0002:0000202c       $unwind$__scrt_fastfail    000000018000d02c     MSVCRT:utility_desktop.obj
 0002:0000203c       $unwind$__isa_available_init 000000018000d03c     MSVCRT:cpu_disp.obj
 0002:00002050       $xdatasym                  000000018000d050     MSVCRT:guard_dispatch.obj
 0002:00002058       $xdatasym                  000000018000d058     MSVCRT:guard_xfg_dispatch.obj
 0002:00002060       .edata                     000000018000d060     nio.exp
 0002:00002088       rgpv                       000000018000d088     nio.exp
 0002:000023bc       rgszName                   000000018000d3bc     nio.exp
 0002:000026f0       rgwOrd                     000000018000d6f0     nio.exp
 0002:0000288a       szName                     000000018000d88a     nio.exp
 0002:00002892       $N00001                    000000018000d892     nio.exp
 0002:0000289d       $N00002                    000000018000d89d     nio.exp
 0002:000028cd       $N00003                    000000018000d8cd     nio.exp
 0002:000028fd       $N00004                    000000018000d8fd     nio.exp
 0002:0000292a       $N00005                    000000018000d92a     nio.exp
 0002:00002954       $N00006                    000000018000d954     nio.exp
 0002:0000297d       $N00007                    000000018000d97d     nio.exp
 0002:000029a7       $N00008                    000000018000d9a7     nio.exp
 0002:000029d1       $N00009                    000000018000d9d1     nio.exp
 0002:000029fc       $N00010                    000000018000d9fc     nio.exp
 0002:00002a36       $N00011                    000000018000da36     nio.exp
 0002:00002a64       $N00012                    000000018000da64     nio.exp
 0002:00002a8e       $N00013                    000000018000da8e     nio.exp
 0002:00002ac1       $N00014                    000000018000dac1     nio.exp
 0002:00002aeb       $N00015                    000000018000daeb     nio.exp
 0002:00002b17       $N00016                    000000018000db17     nio.exp
 0002:00002b40       $N00017                    000000018000db40     nio.exp
 0002:00002b68       $N00018                    000000018000db68     nio.exp
 0002:00002ba2       $N00019                    000000018000dba2     nio.exp
 0002:00002bcc       $N00020                    000000018000dbcc     nio.exp
 0002:00002bf7       $N00021                    000000018000dbf7     nio.exp
 0002:00002c20       $N00022                    000000018000dc20     nio.exp
 0002:00002c4a       $N00023                    000000018000dc4a     nio.exp
 0002:00002c76       $N00024                    000000018000dc76     nio.exp
 0002:00002c9f       $N00025                    000000018000dc9f     nio.exp
 0002:00002ccd       $N00026                    000000018000dccd     nio.exp
 0002:00002cf6       $N00027                    000000018000dcf6     nio.exp
 0002:00002d25       $N00028                    000000018000dd25     nio.exp
 0002:00002d52       $N00029                    000000018000dd52     nio.exp
 0002:00002d7c       $N00030                    000000018000dd7c     nio.exp
 0002:00002da6       $N00031                    000000018000dda6     nio.exp
 0002:00002dd1       $N00032                    000000018000ddd1     nio.exp
 0002:00002dee       $N00033                    000000018000ddee     nio.exp
 0002:00002e17       $N00034                    000000018000de17     nio.exp
 0002:00002e34       $N00035                    000000018000de34     nio.exp
 0002:00002e51       $N00036                    000000018000de51     nio.exp
 0002:00002e70       $N00037                    000000018000de70     nio.exp
 0002:00002e8e       $N00038                    000000018000de8e     nio.exp
 0002:00002eb1       $N00039                    000000018000deb1     nio.exp
 0002:00002ed1       $N00040                    000000018000ded1     nio.exp
 0002:00002eef       $N00041                    000000018000deef     nio.exp
 0002:00002f10       $N00042                    000000018000df10     nio.exp
 0002:00002f2c       $N00043                    000000018000df2c     nio.exp
 0002:00002f58       $N00044                    000000018000df58     nio.exp
 0002:00002f7d       $N00045                    000000018000df7d     nio.exp
 0002:00002fac       $N00046                    000000018000dfac     nio.exp
 0002:00002fc9       $N00047                    000000018000dfc9     nio.exp
 0002:00002ff9       $N00048                    000000018000dff9     nio.exp
 0002:00003024       $N00049                    000000018000e024     nio.exp
 0002:00003050       $N00050                    000000018000e050     nio.exp
 0002:00003081       $N00051                    000000018000e081     nio.exp
 0002:000030b4       $N00052                    000000018000e0b4     nio.exp
 0002:000030e7       $N00053                    000000018000e0e7     nio.exp
 0002:0000311a       $N00054                    000000018000e11a     nio.exp
 0002:00003151       $N00055                    000000018000e151     nio.exp
 0002:00003184       $N00056                    000000018000e184     nio.exp
 0002:000031ba       $N00057                    000000018000e1ba     nio.exp
 0002:000031eb       $N00058                    000000018000e1eb     nio.exp
 0002:0000321f       $N00059                    000000018000e21f     nio.exp
 0002:00003253       $N00060                    000000018000e253     nio.exp
 0002:0000326e       $N00061                    000000018000e26e     nio.exp
 0002:0000328c       $N00062                    000000018000e28c     nio.exp
 0002:000032a6       $N00063                    000000018000e2a6     nio.exp
 0002:000032ca       $N00064                    000000018000e2ca     nio.exp
 0002:000032ee       $N00065                    000000018000e2ee     nio.exp
 0002:0000331e       $N00066                    000000018000e31e     nio.exp
 0002:00003349       $N00067                    000000018000e349     nio.exp
 0002:00003384       $N00068                    000000018000e384     nio.exp
 0002:000033a1       $N00069                    000000018000e3a1     nio.exp
 0002:000033c0       $N00070                    000000018000e3c0     nio.exp
 0002:000033e2       $N00071                    000000018000e3e2     nio.exp
 0002:00003404       $N00072                    000000018000e404     nio.exp
 0002:00003426       $N00073                    000000018000e426     nio.exp
 0002:00003442       $N00074                    000000018000e442     nio.exp
 0002:0000346f       $N00075                    000000018000e46f     nio.exp
 0002:00003494       $N00076                    000000018000e494     nio.exp
 0002:000034be       $N00077                    000000018000e4be     nio.exp
 0002:000034de       $N00078                    000000018000e4de     nio.exp
 0002:000034fe       $N00079                    000000018000e4fe     nio.exp
 0002:00003519       $N00080                    000000018000e519     nio.exp
 0002:0000353e       $N00081                    000000018000e53e     nio.exp
 0002:0000355c       $N00082                    000000018000e55c     nio.exp
 0002:00003575       $N00083                    000000018000e575     nio.exp
 0002:00003595       $N00084                    000000018000e595     nio.exp
 0002:000035b7       $N00085                    000000018000e5b7     nio.exp
 0002:000035d8       $N00086                    000000018000e5d8     nio.exp
 0002:000035f9       $N00087                    000000018000e5f9     nio.exp
 0002:00003619       $N00088                    000000018000e619     nio.exp
 0002:0000363b       $N00089                    000000018000e63b     nio.exp
 0002:0000365c       $N00090                    000000018000e65c     nio.exp
 0002:00003682       $N00091                    000000018000e682     nio.exp
 0002:000036a1       $N00092                    000000018000e6a1     nio.exp
 0002:000036bd       $N00093                    000000018000e6bd     nio.exp
 0002:000036df       $N00094                    000000018000e6df     nio.exp
 0002:00003701       $N00095                    000000018000e701     nio.exp
 0002:00003723       $N00096                    000000018000e723     nio.exp
 0002:00003758       $N00097                    000000018000e758     nio.exp
 0002:0000378c       $N00098                    000000018000e78c     nio.exp
 0002:000037a9       $N00099                    000000018000e7a9     nio.exp
 0002:000037c5       $N00100                    000000018000e7c5     nio.exp
 0002:000037ed       $N00101                    000000018000e7ed     nio.exp
 0002:00003814       $N00102                    000000018000e814     nio.exp
 0002:0000383c       $N00103                    000000018000e83c     nio.exp
 0002:00003864       $N00104                    000000018000e864     nio.exp
 0002:0000388d       $N00105                    000000018000e88d     nio.exp
 0002:000038b7       $N00106                    000000018000e8b7     nio.exp
 0002:000038df       $N00107                    000000018000e8df     nio.exp
 0002:0000390a       $N00108                    000000018000e90a     nio.exp
 0002:00003931       $N00109                    000000018000e931     nio.exp
 0002:00003961       $N00110                    000000018000e961     nio.exp
 0002:0000398b       $N00111                    000000018000e98b     nio.exp
 0002:000039a8       $N00112                    000000018000e9a8     nio.exp
 0002:000039c6       $N00113                    000000018000e9c6     nio.exp
 0002:000039e1       $N00114                    000000018000e9e1     nio.exp
 0002:00003a03       $N00115                    000000018000ea03     nio.exp
 0002:00003a24       $N00116                    000000018000ea24     nio.exp
 0002:00003a48       $N00117                    000000018000ea48     nio.exp
 0002:00003a64       $N00118                    000000018000ea64     nio.exp
 0002:00003aa0       $N00119                    000000018000eaa0     nio.exp
 0002:00003adc       $N00120                    000000018000eadc     nio.exp
 0002:00003b19       $N00121                    000000018000eb19     nio.exp
 0002:00003b5c       $N00122                    000000018000eb5c     nio.exp
 0002:00003ba4       $N00123                    000000018000eba4     nio.exp
 0002:00003be7       $N00124                    000000018000ebe7     nio.exp
 0002:00003c36       $N00125                    000000018000ec36     nio.exp
 0002:00003c78       $N00126                    000000018000ec78     nio.exp
 0002:00003cb6       $N00127                    000000018000ecb6     nio.exp
 0002:00003cf3       $N00128                    000000018000ecf3     nio.exp
 0002:00003d2e       $N00129                    000000018000ed2e     nio.exp
 0002:00003d6d       $N00130                    000000018000ed6d     nio.exp
 0002:00003db7       $N00131                    000000018000edb7     nio.exp
 0002:00003df3       $N00132                    000000018000edf3     nio.exp
 0002:00003e2e       $N00133                    000000018000ee2e     nio.exp
 0002:00003e65       $N00134                    000000018000ee65     nio.exp
 0002:00003e9a       $N00135                    000000018000ee9a     nio.exp
 0002:00003ed4       $N00136                    000000018000eed4     nio.exp
 0002:00003f08       $N00137                    000000018000ef08     nio.exp
 0002:00003f46       $N00138                    000000018000ef46     nio.exp
 0002:00003f83       $N00139                    000000018000ef83     nio.exp
 0002:00003fc1       $N00140                    000000018000efc1     nio.exp
 0002:00003ff2       $N00141                    000000018000eff2     nio.exp
 0002:00004026       $N00142                    000000018000f026     nio.exp
 0002:00004064       $N00143                    000000018000f064     nio.exp
 0002:000040a3       $N00144                    000000018000f0a3     nio.exp
 0002:000040d7       $N00145                    000000018000f0d7     nio.exp
 0002:00004110       $N00146                    000000018000f110     nio.exp
 0002:00004144       $N00147                    000000018000f144     nio.exp
 0002:00004178       $N00148                    000000018000f178     nio.exp
 0002:000041b0       $N00149                    000000018000f1b0     nio.exp
 0002:000041ef       $N00150                    000000018000f1ef     nio.exp
 0002:0000422b       $N00151                    000000018000f22b     nio.exp
 0002:0000425f       $N00152                    000000018000f25f     nio.exp
 0002:000042a6       $N00153                    000000018000f2a6     nio.exp
 0002:000042e7       $N00154                    000000018000f2e7     nio.exp
 0002:00004320       $N00155                    000000018000f320     nio.exp
 0002:00004352       $N00156                    000000018000f352     nio.exp
 0002:00004389       $N00157                    000000018000f389     nio.exp
 0002:000043c0       $N00158                    000000018000f3c0     nio.exp
 0002:000043f9       $N00159                    000000018000f3f9     nio.exp
 0002:0000442f       $N00160                    000000018000f42f     nio.exp
 0002:00004467       $N00161                    000000018000f467     nio.exp
 0002:0000449d       $N00162                    000000018000f49d     nio.exp
 0002:000044cc       $N00163                    000000018000f4cc     nio.exp
 0002:00004507       $N00164                    000000018000f507     nio.exp
 0002:00004541       $N00165                    000000018000f541     nio.exp
 0002:0000457a       $N00166                    000000018000f57a     nio.exp
 0002:000045b4       $N00167                    000000018000f5b4     nio.exp
 0002:000045f0       $N00168                    000000018000f5f0     nio.exp
 0002:00004626       $N00169                    000000018000f626     nio.exp
 0002:00004661       $N00170                    000000018000f661     nio.exp
 0002:0000469e       $N00171                    000000018000f69e     nio.exp
 0002:000046e2       $N00172                    000000018000f6e2     nio.exp
 0002:00004724       $N00173                    000000018000f724     nio.exp
 0002:0000475d       $N00174                    000000018000f75d     nio.exp
 0002:00004793       $N00175                    000000018000f793     nio.exp
 0002:000047d4       $N00176                    000000018000f7d4     nio.exp
 0002:0000480d       $N00177                    000000018000f80d     nio.exp
 0002:00004842       $N00178                    000000018000f842     nio.exp
 0002:0000487b       $N00179                    000000018000f87b     nio.exp
 0002:000048b7       $N00180                    000000018000f8b7     nio.exp
 0002:000048fa       $N00181                    000000018000f8fa     nio.exp
 0002:0000493c       $N00182                    000000018000f93c     nio.exp
 0002:0000497f       $N00183                    000000018000f97f     nio.exp
 0002:000049bb       $N00184                    000000018000f9bb     nio.exp
 0002:000049f9       $N00185                    000000018000f9f9     nio.exp
 0002:00004a34       $N00186                    000000018000fa34     nio.exp
 0002:00004a6a       $N00187                    000000018000fa6a     nio.exp
 0002:00004aaf       $N00188                    000000018000faaf     nio.exp
 0002:00004ae1       $N00189                    000000018000fae1     nio.exp
 0002:00004b1c       $N00190                    000000018000fb1c     nio.exp
 0002:00004b56       $N00191                    000000018000fb56     nio.exp
 0002:00004b94       $N00192                    000000018000fb94     nio.exp
 0002:00004bc8       $N00193                    000000018000fbc8     nio.exp
 0002:00004c01       $N00194                    000000018000fc01     nio.exp
 0002:00004c39       $N00195                    000000018000fc39     nio.exp
 0002:00004c7c       $N00196                    000000018000fc7c     nio.exp
 0002:00004cba       $N00197                    000000018000fcba     nio.exp
 0002:00004cf3       $N00198                    000000018000fcf3     nio.exp
 0002:00004d28       $N00199                    000000018000fd28     nio.exp
 0002:00004d63       $N00200                    000000018000fd63     nio.exp
 0002:00004d9c       $N00201                    000000018000fd9c     nio.exp
 0002:00004dd1       $N00202                    000000018000fdd1     nio.exp
 0002:00004e13       $N00203                    000000018000fe13     nio.exp
 0002:00004e56       $N00204                    000000018000fe56     nio.exp
 0002:00004e8d       $N00205                    000000018000fe8d     nio.exp
 0002:00005696       .idata$6                   0000000180010696     java:java.dll
 0002:0000579c       .idata$6                   000000018001079c     net:net.dll
 0002:00005a10       .idata$6                   0000000180010a10     advapi32:ADVAPI32.dll
 0002:00005a2e       .idata$6                   0000000180010a2e     mswsock:MSWSOCK.dll
 0002:00005a9a       .idata$6                   0000000180010a9a     ws2_32:WS2_32.dll
 0002:000061e4       .idata$6                   00000001800111e4     kernel32:KERNEL32.dll
 0002:00006234       .idata$6                   0000000180011234     vcruntime:VCRUNTIME140.dll
 0002:0000632e       .idata$6                   000000018001132e     ucrt:api-ms-win-crt-heap-l1-1-0.dll
 0002:0000634e       .idata$6                   000000018001134e     ucrt:api-ms-win-crt-string-l1-1-0.dll
 0002:00006370       .idata$6                   0000000180011370     ucrt:api-ms-win-crt-runtime-l1-1-0.dll
 0003:00000000       methods                    0000000180012000     MappedMemoryUtils.obj
 0003:00000060       ?loopback_available@?6??Java_sun_nio_ch_Net_socket0@@9@9 0000000180012060     Net.obj
 0003:00000068       MS_PROVIDER_ID             0000000180012068     UnixDomainSockets.obj
 0003:000001b0       afd__device_name           00000001800121b0     wepoll.obj
 0003:000001c0       afd__device_attributes     00000001800121c0     wepoll.obj
 0003:00000230       handle_fdID                0000000180012230     IOUtil.obj
 0003:00000238       fd_fdID                    0000000180012238     IOUtil.obj
 0003:00000240       completionStatus_error     0000000180012240     Iocp.obj
 0003:00000248       completionStatus_bytesTransferred 0000000180012248     Iocp.obj
 0003:00000250       completionStatus_completionKey 0000000180012250     Iocp.obj
 0003:00000258       completionStatus_overlapped 0000000180012258     Iocp.obj
 0003:00000260       ?handle_fdID@?3??MappedMemoryUtils_force0@@9@9 0000000180012260     MappedMemoryUtils.obj
 0003:00000268       isa_class                  0000000180012268     Net.obj
 0003:00000270       isa_ctorID                 0000000180012270     Net.obj
 0003:00000280       provider                   0000000180012280     UnixDomainSockets.obj
 0003:000004f8       AcceptEx_func              00000001800124f8     WindowsAsynchronousServerSocketChannelImpl.obj
 0003:00000500       ConnectEx_func             0000000180012500     WindowsAsynchronousSocketChannelImpl.obj
 0003:00000508       findFirst_handle           0000000180012508     WindowsNativeDispatcher.obj
 0003:00000510       findFirst_name             0000000180012510     WindowsNativeDispatcher.obj
 0003:00000518       findFirst_attributes       0000000180012518     WindowsNativeDispatcher.obj
 0003:00000520       findStream_handle          0000000180012520     WindowsNativeDispatcher.obj
 0003:00000528       findStream_name            0000000180012528     WindowsNativeDispatcher.obj
 0003:00000530       volumeInfo_fsName          0000000180012530     WindowsNativeDispatcher.obj
 0003:00000538       volumeInfo_volName         0000000180012538     WindowsNativeDispatcher.obj
 0003:00000540       volumeInfo_volSN           0000000180012540     WindowsNativeDispatcher.obj
 0003:00000548       volumeInfo_flags           0000000180012548     WindowsNativeDispatcher.obj
 0003:00000550       diskSpace_bytesAvailable   0000000180012550     WindowsNativeDispatcher.obj
 0003:00000558       diskSpace_totalBytes       0000000180012558     WindowsNativeDispatcher.obj
 0003:00000560       diskSpace_totalFree        0000000180012560     WindowsNativeDispatcher.obj
 0003:00000568       diskSpace_bytesPerSector   0000000180012568     WindowsNativeDispatcher.obj
 0003:00000570       account_domain             0000000180012570     WindowsNativeDispatcher.obj
 0003:00000578       account_name               0000000180012578     WindowsNativeDispatcher.obj
 0003:00000580       account_use                0000000180012580     WindowsNativeDispatcher.obj
 0003:00000588       aclInfo_aceCount           0000000180012588     WindowsNativeDispatcher.obj
 0003:00000590       completionStatus_error     0000000180012590     WindowsNativeDispatcher.obj
 0003:00000598       completionStatus_bytesTransferred 0000000180012598     WindowsNativeDispatcher.obj
 0003:000005a0       completionStatus_completionKey 00000001800125a0     WindowsNativeDispatcher.obj
 0003:000005a8       pGetFileInformationByName  00000001800125a8     WindowsNativeDispatcher.obj
 0003:000005b0       ?zerotime@?1??Java_sun_nio_ch_WindowsSelectorImpl_00024SubSelector_poll0@@9@9 00000001800125b0     WindowsSelectorImpl.obj
 0003:000005c0       NtCancelIoFileEx           00000001800125c0     wepoll.obj
 0003:000005c8       NtCreateFile               00000001800125c8     wepoll.obj
 0003:000005d0       NtCreateKeyedEvent         00000001800125d0     wepoll.obj
 0003:000005d8       NtDeviceIoControlFile      00000001800125d8     wepoll.obj
 0003:000005e0       NtReleaseKeyedEvent        00000001800125e0     wepoll.obj
 0003:000005e8       NtWaitForKeyedEvent        00000001800125e8     wepoll.obj
 0003:000005f0       RtlNtStatusToDosError      00000001800125f0     wepoll.obj
 0003:000005f8       epoll__handle_tree         00000001800125f8     wepoll.obj
 0003:00000608       init__done                 0000000180012608     wepoll.obj
 0003:00000610       init__once                 0000000180012610     wepoll.obj
 0003:00000618       reflock__keyed_event       0000000180012618     wepoll.obj
 0003:00000620       GS_ExceptionRecord         0000000180012620     MSVCRT:gs_report.obj
 0003:000006c0       GS_ContextRecord           00000001800126c0     MSVCRT:gs_report.obj
 0003:00000b90       ?__proc_attached@@3HA      0000000180012b90     MSVCRT:dll_dllmain.obj
 0003:00000bd0       ?is_initialized_as_dll@@3_NA 0000000180012bd0     MSVCRT:utility.obj
 0003:00000bd1       ?module_local_atexit_table_initialized@@3_NA 0000000180012bd1     MSVCRT:utility.obj
 0003:00000bd8       ?module_local_atexit_table@@3U_onexit_table_t@@A 0000000180012bd8     MSVCRT:utility.obj
 0003:00000bf0       ?module_local_at_quick_exit_table@@3U_onexit_table_t@@A 0000000180012bf0     MSVCRT:utility.obj
 0005:00000060       $R000000                   0000000180014060     nio.dll.res
